:106B8400011F0000090101240200000301FA0400AE
:106B9400FA0500030A0A5A0B001E0C00FA0D000342
:106BA4000E00040F0164100096120132130AFA1445
:106BB400010215000017010A1801FA1905321A0119
:106BC4000A1B01FA1C05321FFFFF20FFFF23011ED1
:106BD4002400642A00FA2B00FA2C50782D003D2E54
:106BE40000462F001E3000643250783300003432E7
:106BF400FA350164360164370150380A643C006494
:106C04003E003C3F000140FFFF411450420A5A43FA
:106C14000AC84405324500B44600FA470124480234
:106C2400024C00FA4EFFFF500C0C510596520A32EA
:106C3400530B46540A965602025705465800025909
:106C44000A465A32FA5B010A5C0A325E000A5F00A5
:106C5400FE61FFFF64021066000167FFFF6A0A3CE1
:106C64006B00006C32967300007400007801327976
:106C740001327E00FE7FFFFF80FFFF810000840061
:106C8400FE8500AF8600018700FA8901048A0000AE
:106C94009900009D0A969E00019FFFFFA0FFFFFA46
:106CA400FAFA0065006F00790083008D009700A157
:106CB40000AC00B600C000CA00D400DE00E800F258
:106CC4000058006000680070007800800088009020
:106CD400009800A000A800B000B800C100C800D00F
:106CE40000D800DF00E600EE00F600410047004D4A
:106CF40000530059005F0065006C00710077007D4F
:106D040000830089008F0095009B00A200A700ACBF
:106D140000B200B900C000C500CA00D200D500DD31
:066D240000E100E700EFB2
:103A39009007D6E0FEA3E0FF906B86126E63E493D5
:103A4900F599906B84E493FC740193FDEFB5050738
:103A5900EEB50403754C009007D6126E4A2275A77D
:103A69001085F97285FA737E017F00E573126E3C49
:103A7900E5722FFF50010E8E598F5A900023E0FCFA
:103A8900A3E0FDEF2DFDEE3CFC8C5B8D5C22E55C3B
:103A9900F5FBE55BF5FCD29322E55CF5E9E55BF521
:103AA900EAD29422E55CF5EBE55BF5ECD29122E5EF
:103AB9005CF5EDE55BF5EED29222E55CF5FDE55BA3
:103AC900F5FED28722E55CF5CEE55BF5CFD29022F3
:103AD900AE59AF5A740A8E048F05FF126E2C8C5B97
:103AE9008D5CAE59AF5A740A8E048F05FF126E575A
:103AF9008C598D5AE55A45596013740AC3955AFF72
:103B0900E49559FE8E598F5A785B126E90E572A82A
:103B19005BB80015D3955C4010E572C3955CFFE472
:103B2900955BFE8E5B8F5C8010E5722424C3955CE7
:103B3900FFE4955BFE8E5B8F5CAE5BAF5C74236FBD
:103B49004E600674246F4E701AAE5BAF5C74236FBF
:103B59004E70057572018003757202755C22755B82
:103B6900008003757200229000A6E0B40104C20A25
:103B79008002D20A9000A7E0B40104C20B8002D2ED
:103B89000B9000E4E075F0E1A4FFAEF0740A8E0436
:103B99008F05FF126E2C9007CCECF0A3EDF0A20775
:103BA900401674038C068D07126E3C74011200399D
:103BB9009007CAEEF0A3EFF07E017F009000A2E02B
:103BC900126E3C9000E5E08E048F05FF126E2C7496
:103BD9000AFF126E2C8D5F9000EEE075F0E1A4FFF4
:103BE900AEF0740A8E048F05FF126E2C9007D0EC8C
:103BF900F0A3EDF09000F0E060139000F0E0F5F034
:103C0900741684FF7E00EF9007DEF08006746490DE
:103C190007DEF09000E6E090008AF0900130E09035
:103C29000074F09000E8E0900077F0900094E09044
:103C39000078F09000DAE0900079F090011AE090B5
:103C4900007DF090017EE090007EF090017FE09091
:103C5900007FF0900180E0900080F0A225B340162B
:103C690090017EE0700C90017FE07006900180E089
:103C790060028002C22574E3900089F09000CFE0D1
:103C8900B40B0874E3900089F0805A9000CFE0B437
:103C990019129000E5E0906C9112008CE493900069
:103CA90089F080419000CFE0B41E129000E5E090C9
:103CB9006CAF12008CE493900089F080289000CFBB
:103CC900E0B428129000E5E0906CD912008CE493DE
:103CD900900089F0800F9000CFE0B446089000C6AC
:103CE900E0900089F09000FFE0FE9000CDE06E606A
:103CF9000A9000CDE09000FFF0D22490008DE0FE04
:103D09009000CCE0B5062790008EE0FE9000F8E028
:103D1900B5061B90008FE0FE9000EAE0B5060F9013
:103D29000090E0FE90009FE06E7003023E967404DE
:103D390090011BF090009FE0B40106740090009F71
:103D4900F090009FE0B4020674009000EAF0900041
:103D59009FE0B4030674009000F7F09000F8E0B417
:103D6900012674009000B3F0741C90011EF07400D9
:103D79009006E0F074009006E1F09000CCE0600657
:103D890074009000CCF080329000CCE0601A741C72
:103D99009000B3F0740090011EF074009006E0F0FA
:103DA90074009006E1F08012740090011EF0740016
:103DB9009000B3F0741C9006E0F09000EAE0D39410
:103DC90001402774009000B4F0741B90011DF07439
:103DD900009006DCF074009006DDF09000CCE0B4B1
:103DE900020674019000CCF080339000CCE0B4025C
:103DF9001A741B9000B4F0740090011DF0740090C7
:103E090006DCF074009006DDF0801274009000B4B6
:103E1900F0740090011DF0741B9006DCF09000BF57
:103E2900E060147409900122F074009006E4F074C3
:103E3900009006E5F0800C7400900122F07409905E
:103E490006E4F0D2249000CCE090008DF09000F8C8
:103E5900E090008EF09000EAE090008FF090009FD3
:103E6900E0900090F090009FE0900075F09000BF06
:103E7900E0900076F09000F8E090007AF09000CCA5
:103E8900E090007BF09000EAE090007CF0900091D7
:103E9900E0FE9000BFE06E603E9000BFE0600E74EF
:103EA90009900122F074009006E4F0800C740090EF
:103EB9000122F074099006E4F0900091E060069008
:103EC90000BFE07002D2249000BFE0900091F09012
:103ED90000BFE0900076F0900102E0B40117900075
:103EE9002F740FF0A374FFF0900031E4F0A3F07485
:103EF90002900102F0900102E0B40341900031E028
:103F0900FEA3E0FF90002FE0FCA3E0FD126E887491
:103F190010126E3C7408120039EF900086F0EF70B1
:103F29000674FF900086F07400900102F090003052
:103F3900E0900087F090002FE0900088F0900093C7
:103F4900E090004BF090004BE0240690004CF0907C
:103F5900004BE0240C90004DF090004BE0241290AF
:103F6900004EF090004BE0241890004FF090004B69
:103F7900E0241E900050F090004CE0D39424400BB4
:103F890090004CE0C3942490004CF090004DE0D395
:103F99009424400B90004DE0C3942490004DF09080
:103FA900004EE0D39424400B90004EE0C39424903B
:103FB900004EF090004FE0D39424400B90004FE066
:103FC900C3942490004FF0900050E0D39424400B08
:103FD900900050E0C39424900050F0900057E4F012
:103FE90090004BE06423600790004BE0B4242090DC
:103FF900004BE0B423067402900057F090004BE0A8
:10400900B424069000577401F090004B7401F090AD
:104019000058E4F090004CE06423600790004CE005
:10402900B4242090004CE0B423067402900058F0A8
:1040390090004CE0B424069000587401F090004CB4
:104049007401F0900059E4F090004DE0642360079A
:1040590090004DE0B4242090004DE0B42306740292
:10406900900059F090004DE0B42406900059740175
:10407900F090004D7401F090005AE4F090004EE089
:104089006423600790004EE0B4242090004EE0B411
:104099002306740290005AF090004EE0B424069072
:1040A900005A7401F090004E7401F090005BE4F046
:1040B90090004FE06423600790004FE0B424209003
:1040C900004FE0B42306740290005BF090004FE0CB
:1040D900B4240690005B7401F090004F7401F090D5
:1040E900005CE4F0900050E064236007900050E029
:1040F900B42420900050E0B42306740290005CF0D0
:10410900900050E0B4240690005C7401F0900050D7
:104119007401F0900093E0FE9000F6E02E90005EAE
:10412900F090005EE06412600790005EE0B424063F
:1041390090005EE004F090005EE06411600790007A
:104149005EE0B4230690005EE014F090005EE0D3D8
:104159009424400B90005EE0C3942490005EF0909C
:10416900005EE0D39412400D90005EE0C39412907B
:10417900005FF0800A90005EE0241290005FF07505
:1041890050129000D9E0900051F0900051E075F084
:104199000684AFF07E00EF4E7006900051E004F007
:1041A900900051E00475F00684AFF07E00EF4E7088
:1041B90006900051E014F0900051E0B425069000FB
:1041C900517401F0900051E02406900052F09000E3
:1041D90051E0240C900053F0900051E0241290001B
:1041E90054F0900051E02418900055F0900051E0EF
:1041F900241E900056F0900052E0D39424400B9076
:104209000052E0C39424900052F0900053E0D394FC
:1042190024400B900053E0C39424900053F0900085
:1042290054E0D39424400B900054E0C394249000AC
:1042390054F0900055E0D39424400B900055E0C30E
:104249009424900055F0900056E0D39424400B90AC
:104259000056E0C39424900056F022C293C294C23F
:1042690091C292C287C290E5B554EFF5B5E5B55450
:10427900DFF5B5C296C295C2A0C297C2A2C2A1E596
:10428900B554BFF5B5E5B5547FF5B5E5B554FBF5BE
:10429900B5C20C755D469000DCE07005756C028056
:1042A90003756C0375540075530090001874FFF082
:1042B900A374DCF0C212C214C216C218C21AC21CFC
:1042C90074C8900033F074C8900037F074C8900037
:1042D9003BF074C890003FF074C8900043F074C874
:1042E900900047F0755200755100C207754500E509
:1042F9006EB40903756E00756200900025E4F0A3A1
:10430900F0756F10C20FC210C2119007CCE0FEA366
:10431900E0FF7403126E3C74011200399007CAEE73
:10432900F0A3EFF0C20275560075550090001CE429
:10433900F0A3F0C22675580075570090009EE075ED
:10434900F032A4FDACF090002DECF0A3EDF0C236F4
:10435900A229B39204A22AB39205A22BB3920622F0
:1043690075A71085F97285FA737E017F00E57312CE
:104379006E3CE5722FFF50010E8E598F5AAC5BAD22
:104389005CEF2DFDEE3CFC8C5B8D5CD293D294D21C
:1043990091D292D287D290E55CF5FBE55BF5FCE51D
:1043A9005CF5E9E55BF5EAE55CF5EBE55BF5ECE584
:1043B9005CF5EDE55BF5EEE55CF5FDE55BF5FEE548
:1043C9005CF5CEE55BF5CF75A7002285F97285FA14
:1043D900737E017F00E573126E3CE5722FFF500179
:1043E9000E8E598F5A7E017F76900117E0126E3C2E
:1043F900AC59AD5AED2FFFEC3EFE8E5B8F5CE55C50
:10440900F5E9E55BF5EA90008AE4F0741290006141
:10441900F02285F97285FA737E017F00E573126EC9
:104429003CE5722FFF50010E8E598F5A9007CCE050
:10443900FCA3E0FDEF2DFDEE3CFC8C5B8D5CE55CA7
:10444900F5FBE55BF5FC22056322A2D8B3400CC25B
:1044590096C295C2A0C297C2A2C2A1A2D9B340086E
:104469009000E6E090008AF075D8402285A7717522
:10447900A710A2D8B34002C293A2D9B34002C294F2
:10448900A2DAB34002C291A2DBB34002C292A2DC1B
:10449900B34002C287A2DDB34002C29075D84085FD
:1044A90071A722900047E4936406600280FE74C8F5
:1044B9009007D2F8E4F0E8A3F075B50075840175AA
:1044C900A70075FFA090005DE4F075C91075A70FEE
:1044D90075A1C775A70075D90075CE0C75A70F759D
:1044E900F1FE75F2FF75F30775F47875A4BA75A531
:1044F900FF75A60775AE0075AFFF75D48175D5FF39
:1045090075D6FF75D7FF75A70075A20175A1477507
:10451900F80975D80075D90475DA0975DB0975D8F4
:104529004075A71075D80075D90475DA0975DB09C6
:1045390075DC0975DD0975DE0975DF0975D8407502
:10454900A70075E60875E71075BC0175BE0475BD51
:104559006C75BE0775BDA075BE0875BD0175BC003B
:1045690075BB1875BC2075BA0875E88075D11375C7
:10457900A70F75E10575E20075C74012426475978A
:1045890000759780740A126E1C7597C0E5975420C0
:10459900700280F8758F0275A700D2AF7598007503
:1045A900A90C75A70F75AB4375ADFB75AC1E75A747
:1045B9001075C91875CA0075CB0075C80475A700B0
:1045C900758912758E04758C00758A00C2A9D28C02
:1045D900758D00758B00D2ABD28E75EF0675D944F7
:1045E900C29974C8F5097508001200E975B5001279
:1045F90004E974639007D2F8E4F0E8A3F0120375B4
:1046090074C89007D2F8E4F0E8A3F07464F509756A
:1046190008001200E9900075E090009FF090009F5B
:10462900E0D39403400C740090009FF07400900054
:1046390075F0C22090009FE090678CF8282873805D
:1046490028A2B44002D220802075A70F75F30F75F8
:10465900A700A2A34002D220800F75A70F75F317F8
:0946690075A700A2A44002D220B2
:0C678C0002464802464A0246520246639A
:10467200A220B3405F757208E572D3940E5020E514
:10468200729007D2F8E4F0E8A3F01202447464F5E1
:10469200097508001200E97872740126F650D9747F
:1046A200029000DBF0900075E090009FF090009F78
:1046B200E0906798F828287380167400900105F03E
:1046C200800E74009000EAF0800674009000F7F00B
:0C6798000246BA0246BC0246C40246CCCF
:1046D200D21F805D757201E572D394075020E57296
:1046E2009007D2F8E4F0E8A3F01202447464F509EA
:1046F2007508001200E97872740126F650D9740127
:104702009000DBF0900075E090009FF090009FE039
:104712009067A4F828287380167400900105F08031
:0F4722000E74009000EAF0800674009000F7F02B
:0C67A40002471902471B02472302472B43
:10473100C21F900074E0900130F0900075E090008D
:104741009FF0900076E09000BFF0900077E090003D
:10475100E8F0900078E0900094F0900079E090000B
:10476100DAF090007AE09000F8F090007BE09000A1
:10477100CCF090007CE09000EAF090007DE09001A8
:104781001AF090007EE090017EF090007FE09001B1
:104791007FF0900080E0900180F090017EE0700C4D
:1047A10090017FE07006900180E060028004C225E4
:1047B1008002D2259000E5E07006740A9000E5F0D1
:1047C1009000C6E0700674E39000C6F09000CCE063
:1047D1000490008DF09000BFE004900091F09000F3
:1047E100CDE09000FFF0123B70E5B54401F5B574E2
:1047F10006900063F07401900064F0740390006609
:10480100F07405900067F0743B900068F0740690B6
:104811000069F0740190006AF0740090006FF07408
:1048210000900072F074FF900073F074339001698E
:10483100F0743690016AF0742D90016BF07432902F
:10484100016CF0742090016DF0744C90016EF07465
:104851006590016FF07478900170F074759001713A
:10486100F07473900172F07420900173F07456909B
:104871000174F07431900175F07432900176F07426
:1048810020900177F0900101E0900086F09000B84F
:10489100E0900087F09000B9E0900088F0A2B6B3F4
:1048A1009208A2B3B39209A2A4B39222A2A3B39293
:1048B10023900082E4F0756E00743A900792F074D0
:1048C100FD900793F0900083E4F09007CCE0FEA305
:1048D100E0FF7403126E3C74011200399007CAEEB6
:1048E100F0A3EFF0756D01900061E4F0C2217562F3
:1048F10000C20DD20EC202757000C228D203C229B5
:10490100D204C22AD205C22412009E755E00756AC5
:104911000075600075643275650075660075670025
:10492100756800756900900025E4F0A3F0756B00CF
:10493100D2B2D2A4D2B0D2B1D2A3D2A7D2A6D2A59A
:10494100D2B790009EE0D394FA400674FA90009E8C
:10495100F07E017F00900088E0126E3C900087E0BD
:104961002FFF50010E90002FEEF0A3EFF0EFD39444
:10497100FFEE940F400790002FE4F0A3F090008623
:10498100E0700674FF900086F09000DBE0D39402A3
:10499100400674019000DBF09000DCE07005756C5E
:1049A100028003756C039000DDE0D394014006742E
:1049B100009000DDF09000E3E0C3940A5006740A11
:1049C1009000E3F09000EDE0700674019000EDF0CE
:1049D1009000EDE0B4FF0674FE9000EDF09000F45D
:1049E100E0D394FE400674FE9000F4F090011AE0CA
:1049F100D394024006740190011AF0900130E0D383
:104A0100940140067401900130F074019000FAF0B5
:104A110074019000FBF07400900102F074089001A1
:104A21001FF07407900120F0742A900121F074297D
:104A31009006D8F0D29C9000CDE0D3940440067447
:104A4100049000CDF0E56FD394104003756F109082
:104A510006D9E0D3940C400674009006D9F0900674
:104A6100DDE0D3940C400674009006DDF09006E181
:104A7100E0D3940C400674009006E1F09006E5E066
:104A8100D3940C400674009006E5F0D2EC75CF018A
:104A9100A298B34005C298120646E54C6006A29959
:104AA100B3B340028005C299120C57E54D64016011
:104AB10005E54DB4040280D5C28E7E107F00E5630A
:104AC100126E3CE58D75F010A4FDACF0EF2DFDEEFE
:104AD1003CFCE58B75F01084FF7E00ED2FFFEC3E72
:104AE100FE8E538F54D28E9000BFE060099000BFBC
:104AF100E0C3943D40028056900027126E4A900018
:104B010027E0FEA3E0FF900029E0FCA3E0FDEFB564
:104B1100053CEEB50438B21EA207B34013A21EB382
:104B21004008E5B54404F5B58006E5B554FBF5B597
:104B3100900029E0FEA3E0FF90002BE0FCA3E0FD44
:104B4100EF2DFDEE3CFC900029ECF0A3EDF0900080
:104B5100CCE060099000CCE0C394034003024BFC1D
:104B6100122D96A207B35009900082E0C3941F4012
:104B71000280069000B6E0F544E54475F005A4FF17
:104B8100AEF09007D4EEF0A3EFF09000A3E0C39550
:104B9100604007E55EC3955F50079007D4E4F0A33A
:104BA100F0AE2DAF2E9007D4E0FCA3E0FDEFD39D36
:104BB100EE9C4020E5B5547FF5B59000CCE0B40201
:104BC100099000EAE0C3940240028006E5B5444042
:104BD100F5B58027900082E0C3942E5006E5B544D8
:104BE10080F5B59000CCE0B402099000EAE0C394EE
:104BF1000240028006E5B554BFF5B59000CCE0B4A3
:104C01000324122EB1AE2DAF2E9007D4E0FCA3E009
:104C1100FDEFD39DEE9C4008E5B54480F5B58006D7
:104C2100E5B5547FF5B5A2B6300801B35003025281
:104C310030A2B6300801B35003025230A2B6300A96
:104C410001B350030250C1756D009000BFE0B43D47
:104C510013A20AB34008E5B554FBF5B58006E5B5E6
:104C61004404F5B5055DA20CB3B35013AE53AF5474
:104C7100900018E0FCA3E0FDEDC39FEC9E40030211
:104C81004D9EE56CB4032EA226B34022E55DB4230C
:104C910003756C01E55DC3942350069000617401B6
:104CA100F0E55DD3942340067402900061F0755DD8
:104CB10001D2268062E56CB40206756C01755D2334
:104CC100E55DB42305755D01804D900061E07038AC
:104CD100E55DC3942350069000617401F0E55DD356
:104CE100942340067402900061F0E55DC394235063
:104CF10002D221E55DD394234002D221C296C2950E
:104D0100C2A0C297C2A2C2A19000DCE0B401051208
:104D110042648003755D01AE55AF56AC53AD54EF9F
:104D21002DFDEE3CFC74028C068D071200398E5568
:104D31008F569000BFE060099000BFE0C3943D40F2
:104D4100028043900027E0FEA3E0FF9000BFE08EC9
:104D5100048F05FF126E2C74018C068D0712003929
:104D610090002BEEF0A3EFF090002BE0F8A3E09081
:104D71000029C8F0A3C8F0900027E4F0A3F0C21EF8
:104D8100E5B554FBF5B5A2A4B34002C222A2A3B378
:104D91004002C223A221B34002C221803AAE55AFE4
:104DA10056AC53AD54EF2DFDEE3CFC74018C068DD9
:104DB100071200398E558F56E56CC39402500DAC25
:104DC10053AD547488C39D74139C400280091242F0
:104DD100647406900061F0E55DB4231274039000E1
:104DE10061F0D2219000DCE0B40103124264AE57BD
:104DF100AF58AC53AD54EF2DFDEE3CFC8C578D58A4
:104E0100AE53AF54EFD39DEE9C401190001FE0FADA
:104E1100A3E0FBEBC394E8EA940340028006900010
:104E21001F126E4A90001CE0FEA3E0FFAC53AD548C
:104E3100EF2DFDEE3CFC90001CECF0A3EDF090009A
:104E4100DCE0B40118AE53AF547405126E3C74012A
:104E5100120039900018EEF0A3EFF08011AE53AFBD
:104E6100547402126E3C900018EEF0A3EFF0C28E63
:104E7100758D00758B00756300755401755300D2F3
:104E81008EE55D240875F00984AFF07E00EF4E7069
:104E91007590001CE0F8A3E090001AC8F0A3C8F0D8
:104EA10090001AE0FEA3E0FFEF4E600B7C837D06CD
:104EB100126D2A8E518F5290001CE4F0A3F0AE5176
:104EC100AF527428BE00039F5010E5622FFF5001BE
:104ED1000E74011200398E518F528552629000E397
:104EE100E0A851B8000DD395524008E552900060FA
:104EF100F080099000E3E014900060F0E56C60063A
:104F0100755200755100E55D640B6005E55DB41DEA
:104F1100099000CCE060031223D290005EE0655D51
:104F2100600790005FE0B55D03756E00A20DB350A0
:104F310006A20CB3B34003024FE0900098E0B40125
:104F41007390011AE0B40214120E2690008BE075E2
:104F5100F0BEA4FFAEF08E5B8F5C8056E56675F007
:104F61000A84FF7E00900592126E63E0F55A75592E
:104F710000AE59AF5A9000BDE0126E3C74648E04CD
:104F81008F05FF126E2C8C5B8D5CE55C90001EF032
:104F9100AE59AF5A900096E0126E3C74648E048F45
:104FA10005FF126E2C74BE8C068D07126E3C8E5B53
:104FB1008F5C8017900096E075F0BEA4FFAEF08E76
:104FC1005B8F5C9000BDE090001EF0E560C394CC67
:104FD1005006E55C455B70028003124369D20DE522
:104FE1006CB40106E55D640B60028009756F019088
:104FF10000627401F0E56C60030250BC9000DFE0D8
:10500100600D90008AE0A851B800069552400280D8
:10501100409000DFE0B4021F90004BE0655D600F3F
:1050210090004CE0655D600790004DE0B55D037553
:105031006F03756B00800CC200756B00900025E456
:10504100F0A3F090008AE060067409900061F0809E
:105051006A90004BE0B55D0B756F019000627401C1
:10506100F0805890004CE0B55D0B756F01740290B3
:105071000062F0804690004DE0B55D0B756F0174E4
:1050810003900062F0803490004EE0B55D0B756FC7
:10509100017404900062F0802290004FE0B55D0B36
:1050A100756F017405900062F08010900050E0B5BA
:1050B1005D09756F017406900062F0A20AB392084F
:1050C100A20AB330B601B35003025230756D01909C
:1050D10000BFE0B43D13A20AB34008E5B54404F5AE
:1050E100B58006E5B554FBF5B5E5B54401F5B574F4
:1050F1001F900082F0A20A9208E55DD3944A401401
:10510100D20CE55DD3946D400B7404900061F0D234
:1051110021755D469000E7E0B40107E569C3941489
:10512100400280091242647413900061F0A2283099
:105131000301B35017A228B34008E5B54408F5B5FB
:105141008006E5B554F7F5B5A2289203A2293004EB
:1051510001B35017A229B34008E5B54440F5B58025
:1051610006E5B554BFF5B5A2299204A22A3005017E
:10517100B35017A22AB34008E5B54480F5B58006BF
:10518100E5B5547FF5B5A22A9205A22B300601B3ED
:105191005017A22BB34008E5B54404F5B58006E5E8
:1051A100B554FBF5B5A22B9206900115E0A851B8B4
:1051B1000005D39552500D900114E0A851B8000498
:1051C100955250028008E5B54402F5B5801790016B
:1051D10016E0D395604008E5B54402F5B58006E5D3
:1051E100B554FDF5B5E569C394415009740E9000BD
:1051F10061F0124264900069E0FE900065E0C39E98
:105201004009900065E0D39408400974FB90006167
:10521100F012426490006EE0601590006EE0FE9026
:105221000068E06E600974FE900061F0124264A2B1
:1052310021B3400CC296C295C2A0C297C2A2C2A11C
:10524100900117E0600CAE51AF527414BE00059F7F
:105251004002803790009FE09067B0F82828738063
:105261002A8028A2A3B35005A223B34002800512CD
:1052710043D4D2238015A2A4B35005A222B3400285
:0B52810080051243D4D222800280007E
:1067B00002526002526202526402527702528A020C
:0267C000528CF9
:10528C00A20FB3B35008900051E0655D6002803608
:10529C00A201B35006A200B3B340028023123A67B6
:1052AC00123A979000F8E0B40113A202B34008E55B
:1052BC00B54480F5B58006E5B5547FF5B575A70006
:1052CC00C20FD210D211A210B3B35008900052E00A
:1052DC00655D60028036A201B35006A200B3B340F4
:1052EC00028023123A67123AA29000F8E0B401133C
:1052FC00A202B34008E5B54480F5B58006E5B55487
:10530C007FF5B575A700D20FC210D211A211B3B39D
:10531C005008900053E0655D60028036A201B350E6
:10532C0006A200B3B340028023123A67123AAD9042
:10533C0000F8E0B40113A202B34008E5B54480F5CF
:10534C00B58006E5B5547FF5B575A700D20FD21020
:10535C00C211A20FB3B35008900054E0655D600217
:10536C008036A201B35006A200B3B34002802312D0
:10537C003A67123AB89000F8E0B40113A202B340B5
:10538C0008E5B54480F5B58006E5B5547FF5B575EF
:10539C00A700C20FD210D211A210B3B350089000C4
:1053AC0055E0655D60028036A201B35006A200B3E1
:1053BC00B340028023123A67123AC39000F8E0B46B
:1053CC000113A202B34008E5B54480F5B58006E5AB
:1053DC00B5547FF5B575A700D20FC210D211A2112A
:1053EC00B3B35008900056E0655D60028036A201B0
:1053FC00B35006A200B3B340028023123A67123AAC
:10540C00CE9000F8E0B40113A202B34008E5B54415
:10541C0080F5B58006E5B5547FF5B575A700D20FBC
:10542C00D210C211E56F9067C2F8282873025B5046
:04543C009000CDE02F
:0667C20002543902543CB0
:105440009067F5F8282873121EAE8012121EAE80E7
:0E5450000D121F388008121FE48003121FE4A3
:0F67F50002544702544C02545102545602545B52
:10545E00756F02025B50122110122227A236B34042
:10546E00229000C1E0F56B900092E0256BFE90005B
:10547E0060E075F01E84FC7F00EE2CF53574109004
:10548E000061F09007CAE0FEA3E0FF740A126E3CC2
:10549E0090001AE0FCA3E0FD74098F02FF126E2C3F
:1054AE008D078C038E048A058B06126D2A9007CE0B
:1054BE00EEF0A3EFF074F0BE00039F500B74F0906B
:1054CE0007CEF8E4F0E8A3F0E535700375350190EA
:1054DE0007CEE0FEA3E0FFE5352FFF50010E90074B
:0D54EE00CEEEF0A3EFF0756F03900062E0CA
:0367C80002546414
:1054FB00906804F82828738034A2374003756F0A2C
:10550B00802BA2374003756F0B8022A237400375A7
:10551B006F0C8019A2374003756F0D8010A23740B6
:0D552B0003756F0E8007A2374003756F0FE8
:1068040002550202550402550D02551602551F0287
:0568140055280255317A
:10553800025B509006D9E060031224EA900118E05B
:10554800B40114900119E0A851B80004955250070D
:10555800E55EC3955F400280097415900061F00212
:1055680055EB9000CDE0D39402403F9000A1E02499
:1055780003A851B80004955250099000A3E0D395B0
:105588006050028008D2017408900061F09000A178
:10559800E0A851B80005D39552500B9000A3E02421
:1055A80003C395605002C20180399000A1E0240332
:1055B800A851B8000495525007E55EC3955F4002B4
:1055C8008008D2017408900061F09000A1E0A85111
:1055D800B80005D395525009E55F240FC3955E5076
:1055E80002C2019000E7E07007E569C39414400225
:1055F8008002D201A2014005756F04800A756F1000
:10560800900025E4F0A3F0A207B34029E56675F001
:105618000A84FF7E00900592126E63E0C39469507D
:1056280005122407800F9007CCE0F8A3E09007CA82
:0C563800C8F0A3C8F0025B509000CDE069
:0667CB0002553B0256409E
:10564400906819F8282873120F108012120F108016
:0E5654000D1210BE800812117080031211702A
:0F68190002564B02565002565502565A02565F0F
:105662009006DDE060031225C6756F05025B5012DD
:1056720012B0756F069006E1E060031226B6025B77
:105682005090001EE06006A207B3B34002801D9056
:10569200001EE02528FFAE2750010E8E278F28E539
:1056A2005DD39406500690001EE014F01214F675B5
:1056B2006F079006E5E06003122792025B509001AB
:1056C2001AE0B40203120E9E1218F5756F08025BFF
:1056D20050121CB1A20FB35005A210B340028006B3
:1056E200D20FD210D211756F10025B50025B509034
:1056F2000035E0C394465008C2967446900035F0D7
:10570200900057E0B4011DE535240AF5359007CE27
:10571200E0FEA3E0FF740A2FFF50010E9007CEEEC9
:10572200F0A3EFF0900057E0B4021DE5352414F524
:10573200359007CEE0FEA3E0FF74142FFF50010E58
:105742009007CEEEF0A3EFF085355A755900900020
:105752004BE0F572123AD9E55C900035F090000CFE
:10576200E559F0A3E55AF0E572900036F0C21390C5
:1057720007CEE0F559A3E0F55A90004BE0F572121E
:105782003AD9E55C900033F0900000E559F0A3E5CA
:105792005AF0E572900034F0C212E56CB40105755E
:1057A2006F0B8003756F03025B50900039E0C39466
:1057B200465008C2957446900039F0900058E0B403
:1057C200011DE535240AF5359007CEE0FEA3E0FF82
:1057D200740A2FFF50010E9007CEEEF0A3EFF09067
:1057E2000058E0B4021DE5352414F5359007CEE0EB
:1057F200FEA3E0FF74142FFF50010E9007CEEEF0CF
:10580200A3EFF085355A75590090004CE0F57212FD
:105812003AD9E55C900039F090000EE559F0A3E525
:105822005AF0E57290003AF0C2159007CEE0F559B1
:10583200A3E0F55A90004CE0F572123AD9E55C907B
:105842000037F0900002E559F0A3E55AF0E57290B6
:105852000038F0C214E56CB40105756F0C80037555
:105862006F03025B5090003DE0C394465008C2A013
:10587200744690003DF0900059E0B4011DE53524D6
:105882000AF5359007CEE0FEA3E0FF740A2FFF5021
:10589200010E9007CEEEF0A3EFF0900059E0B402B3
:1058A2001DE5352414F5359007CEE0FEA3E0FF7424
:1058B200142FFF50010E9007CEEEF0A3EFF08535C6
:1058C2005A75590090004DE0F572123AD9E55C9094
:1058D200003DF0900010E559F0A3E55AF0E5729012
:1058E200003EF0C2179007CEE0F559A3E0F55A90BA
:1058F200004DE0F572123AD9E55C90003BF0900061
:1059020004E559F0A3E55AF0E57290003CF0C216A6
:10591200E56CB40105756F0D8003756F03025B5072
:10592200900041E0C394465008C2977446900041EB
:10593200F090005AE0B4011DE535240AF5359007D0
:10594200CEE0FEA3E0FF740A2FFF50010E9007CEB7
:10595200EEF0A3EFF090005AE0B4021DE5352414F6
:10596200F5359007CEE0FEA3E0FF74142FFF50013F
:105972000E9007CEEEF0A3EFF085355A75590090E0
:10598200004EE0F572123AD9E55C900041F09000C9
:1059920012E559F0A3E55AF0E572900042F0C219FF
:1059A2009007CEE0F559A3E0F55A90004EE0F5726B
:1059B200123AD9E55C90003FF0900006E559F0A359
:1059C200E55AF0E572900040F0C218E56CB40105AA
:1059D200756F0E8003756F03025B50900045E0C344
:1059E20094465008C2A27446900045F090005BE0D5
:1059F200B4011DE535240AF5359007CEE0FEA3E09B
:105A0200FF740A2FFF50010E9007CEEEF0A3EFF0C5
:105A120090005BE0B4021DE5352414F5359007CE05
:105A2200E0FEA3E0FF74142FFF50010E9007CEEEAC
:105A3200F0A3EFF085355A75590090004FE0F572EA
:105A4200123AD9E55C900045F0900014E559F0A3B4
:105A5200E55AF0E572900046F0C21B9007CEE0F5E1
:105A620059A3E0F55A90004FE0F572123AD9E55C7D
:105A7200900043F0900008E559F0A3E55AF0E57272
:105A8200900044F0C21AE56CB40105756F0F8003F3
:105A9200756F03025B50900049E0C394465008C200
:105AA200A17446900049F090005CE0B4011DE53518
:105AB200240AF5359007CEE0FEA3E0FF740A2FFF1B
:105AC20050010E9007CEEEF0A3EFF090005CE0B430
:105AD200021DE5352414F5359007CEE0FEA3E0FF64
:105AE20074142FFF50010E9007CEEEF0A3EFF08555
:105AF200355A755900900050E0F572123AD9E55CBA
:105B0200900049F0900016E559F0A3E55AF0E572CD
:105B120090004AF0C21D9007CEE0F559A3E0F55A75
:105B2200900050E0F572123AD9E55C900047F0908F
:105B3200000AE559F0A3E55AF0E572900048F0C278
:0E5B42001CE56CB40103756C00756F038000E8
:1067D1000256710256830256C00256D30256EE0289
:1067E10056F10257AC0258670259220259DD025A8A
:0467F10098025B505F
:105B5000900033E0B55D028003025BF2A212407256
:105B6000900000E0FEA3E0FFEF4E6021AE55AF567F
:105B7000900000E0FCA3E0FD120003740A8E048F85
:105B800005FF126E2C900000ECF0A3EDF0900034B5
:105B9000E0601A900000E0FEA3E0FFAC55AD56EFC8
:105BA0002DFDEE3CFC900000ECF0A3EDF0900034F5
:105BB000E0D39401401A900000E0FEA3E0FFAC5552
:105BC000AD56EF2DFDEE3CFC900000ECF0A3EDF0A7
:105BD000D212AE53AF54900000E0FCA3E0FDEFC33F
:105BE0009DEE9C400D12441BD296C21274C89000C8
:105BF00033F0A212B3B35007900033E0B55D0280DA
:105C00000D12441BD29674C8900033F0C21290005B
:105C100035E0B55D028003025CADA21340729000D6
:105C20000CE0FEA3E0FFEF4E6021AE55AF569000B2
:105C30000CE0FCA3E0FD120003740A8E048F05FF44
:105C4000126E2C90000CECF0A3EDF0900036E060AA
:105C50001A90000CE0FEA3E0FFAC55AD56EF2DFD11
:105C6000EE3CFC90000CECF0A3EDF0900036E0D39D
:105C70009401401A90000CE0FEA3E0FFAC55AD5635
:105C8000EF2DFDEE3CFC90000CECF0A3EDF0D213F8
:105C9000AE53AF5490000CE0FCA3E0FDEFC39DEECB
:105CA0009C400AC2967446900035F0C213A213B30A
:105CB000B35007900035E0B55D02800AC296744685
:105CC000900035F0C213900037E0B55D028003020A
:105CD0005D68A2144072900002E0FEA3E0FFEF4E68
:105CE0006021AE55AF56900002E0FCA3E0FD12002B
:105CF00003740A8E048F05FF126E2C900002ECF0E4
:105D0000A3EDF0900038E0601A900002E0FEA3E0FE
:105D1000FFAC55AD56EF2DFDEE3CFC900002ECF0D3
:105D2000A3EDF0900038E0D39401401A900002E017
:105D3000FEA3E0FFAC55AD56EF2DFDEE3CFC900010
:105D400002ECF0A3EDF0D214AE53AF54900002E099
:105D5000FCA3E0FDEFC39DEE9C400D12441BD295C9
:105D6000C21474C8900037F0A214B3B35007900067
:105D700037E0B55D02800D12441BD29574C89000C7
:105D800037F0C214900039E0B55D028003025E2353
:105D9000A215407290000EE0FEA3E0FFEF4E6021DE
:105DA000AE55AF5690000EE0FCA3E0FD1200037468
:105DB0000A8E048F05FF126E2C90000EECF0A3EDFE
:105DC000F090003AE0601A90000EE0FEA3E0FFAC15
:105DD00055AD56EF2DFDEE3CFC90000EECF0A3ED22
:105DE000F090003AE0D39401401A90000EE0FEA338
:105DF000E0FFAC55AD56EF2DFDEE3CFC90000EECF7
:105E0000F0A3EDF0D215AE53AF5490000EE0FCA31A
:105E1000E0FDEFC39DEE9C400AC2957446900039A8
:105E2000F0C215A215B3B35007900039E0B55D027A
:105E3000800AC2957446900039F0C21590003BE08C
:105E4000B55D028003025EDEA2164072900004E09F
:105E5000FEA3E0FFEF4E6021AE55AF56900004E088
:105E6000FCA3E0FD120003740A8E048F05FF126E7E
:105E70002C900004ECF0A3EDF090003CE0601A9050
:105E80000004E0FEA3E0FFAC55AD56EF2DFDEE3C67
:105E9000FC900004ECF0A3EDF090003CE0D3940102
:105EA000401A900004E0FEA3E0FFAC55AD56EF2D84
:105EB000FDEE3CFC900004ECF0A3EDF0D216AE53E6
:105EC000AF54900004E0FCA3E0FDEFC39DEE9C40C6
:105ED0000D12441BD2A0C21674C890003BF0A2164B
:105EE000B3B3500790003BE0B55D02800D12441B38
:105EF000D2A074C890003BF0C21690003DE0B55DA2
:105F0000028003025F99A2174072900010E0FEA386
:105F1000E0FFEF4E6021AE55AF56900010E0FCA3BD
:105F2000E0FD120003740A8E048F05FF126E2C90A0
:105F30000010ECF0A3EDF090003EE0601A9000102D
:105F4000E0FEA3E0FFAC55AD56EF2DFDEE3CFC901E
:105F50000010ECF0A3EDF090003EE0D39401401A65
:105F6000900010E0FEA3E0FFAC55AD56EF2DFDEE26
:105F70003CFC900010ECF0A3EDF0D217AE53AF5400
:105F8000900010E0FCA3E0FDEFC39DEE9C400AC230
:105F9000A0744690003DF0C217A217B3B35007900B
:105FA000003DE0B55D02800AC2A0744690003DF05D
:105FB000C21790003FE0B55D028003026054A21852
:105FC0004072900006E0FEA3E0FFEF4E6021AE5568
:105FD000AF56900006E0FCA3E0FD120003740A8EA9
:105FE000048F05FF126E2C900006ECF0A3EDF090EC
:105FF0000040E0601A900006E0FEA3E0FFAC55AD63
:1060000056EF2DFDEE3CFC900006ECF0A3EDF09079
:106010000040E0D39401401A900006E0FEA3E0FFA8
:10602000AC55AD56EF2DFDEE3CFC900006ECF0A318
:10603000EDF0D218AE53AF54900006E0FCA3E0FDA3
:10604000EFC39DEE9C400D12441BD297C21874C83A
:1060500090003FF0A218B3B3500790003FE0B55D49
:1060600002800D12441BD29774C890003FF0C218F2
:10607000900041E0B55D02800302610FA2194072F9
:10608000900012E0FEA3E0FFEF4E6021AE55AF5648
:10609000900012E0FCA3E0FD120003740A8E048F4E
:1060A00005FF126E2C900012ECF0A3EDF090004270
:1060B000E0601A900012E0FEA3E0FFAC55AD56EF91
:1060C0002DFDEE3CFC900012ECF0A3EDF0900042B0
:1060D000E0D39401401A900012E0FEA3E0FFAC551B
:1060E000AD56EF2DFDEE3CFC900012ECF0A3EDF070
:1060F000D219AE53AF54900012E0FCA3E0FDEFC301
:106100009DEE9C400AC2977446900041F0C219A2CD
:1061100019B3B35007900041E0B55D02800AC29701
:106120007446900041F0C219900043E0B55D0280D2
:10613000030261CAA21A4072900008E0FEA3E0FFC9
:10614000EF4E6021AE55AF56900008E0FCA3E0FD95
:10615000120003740A8E048F05FF126E2C90000843
:10616000ECF0A3EDF0900044E0601A900008E0FE2F
:10617000A3E0FFAC55AD56EF2DFDEE3CFC900008C2
:10618000ECF0A3EDF0900044E0D39401401A9000AD
:1061900008E0FEA3E0FFAC55AD56EF2DFDEE3CFC54
:1061A000900008ECF0A3EDF0D21AAE53AF5490007B
:1061B00008E0FCA3E0FDEFC39DEE9C400D12441BE4
:1061C000D2A2C21A74C8900043F0A21AB3B3500707
:1061D000900043E0B55D02800D12441BD2A274C84A
:1061E000900043F0C21A900045E0B55D02800302C2
:1061F0006285A21B4072900014E0FEA3E0FFEF4E08
:106200006021AE55AF56900014E0FCA3E0FD1200F3
:1062100003740A8E048F05FF126E2C900014ECF0AC
:10622000A3EDF0900046E0601A900014E0FEA3E0B9
:10623000FFAC55AD56EF2DFDEE3CFC900014ECF09C
:10624000A3EDF0900046E0D39401401A900014E0D2
:10625000FEA3E0FFAC55AD56EF2DFDEE3CFC9000EB
:1062600014ECF0A3EDF0D21BAE53AF54900014E049
:10627000FCA3E0FDEFC39DEE9C400AC2A2744690D1
:106280000045F0C21BA21BB3B35007900045E0B518
:106290005D02800AC2A27446900045F0C21B9000C5
:1062A00047E0B55D028003026340A21C407290008B
:1062B0000AE0FEA3E0FFEF4E6021AE55AF5690001E
:1062C0000AE0FCA3E0FD120003740A8E048F05FFB0
:1062D000126E2C90000AECF0A3EDF0900048E06004
:1062E0001A90000AE0FEA3E0FFAC55AD56EF2DFD7D
:1062F000EE3CFC90000AECF0A3EDF0900048E0D3F7
:106300009401401A90000AE0FEA3E0FFAC55AD56A0
:10631000EF2DFDEE3CFC90000AECF0A3EDF0D21C5A
:10632000AE53AF5490000AE0FCA3E0FDEFC39DEE36
:106330009C400D12441BD2A1C21C74C8900047F0AF
:10634000A21CB3B35007900047E0B55D02800D1268
:10635000441BD2A174C8900047F0C21C900049E0D1
:10636000B55D0280030263FBA21D4072900016E03F
:10637000FEA3E0FFEF4E6021AE55AF56900016E051
:10638000FCA3E0FD120003740A8E048F05FF126E59
:106390002C900016ECF0A3EDF090004AE0601A900B
:1063A0000016E0FEA3E0FFAC55AD56EF2DFDEE3C30
:1063B000FC900016ECF0A3EDF090004AE0D39401BD
:1063C000401A900016E0FEA3E0FFAC55AD56EF2D4D
:1063D000FDEE3CFC900016ECF0A3EDF0D21DAE53A8
:1063E000AF54900016E0FCA3E0FDEFC39DEE9C408F
:1063F0000AC2A17446900049F0C21DA21DB3B35059
:1064000007900049E0B55D02800AC2A17446900081
:1064100049F0C21D9000EAE0B40202800302653F29
:10642000900084E0D395655064900084E0F40425E6
:1064300065FE9000EDE08E00F5F0E884FF7E008FB1
:1064400072EFC39410500CEF8572F0A4FDACF08D88
:106450007280037572FF900084E0D39572400B90B8
:106460000084E0C39572F570800375700090010898
:10647000E0D395704006900108E0F570900109E0C6
:10648000C395705006900109E0F57080719000840A
:10649000E0C39565FE9000EDE08E00F5F0E884FF26
:1064A0007E008F72EFC39410500CEF8572F0A4FD44
:1064B000ACF08D7280037572FF85725A7559009029
:1064C0000084E0255AFFAE5950010E8E598F5A7440
:1064D000FFBE0009D39F4005855A7080037570FF89
:1064E000900108E0D395704006900108E0F57090A7
:1064F0000109E0C395705006900109E0F570A2070C
:10650000B3B3500D900085E0FE9000F5E0D39E50AF
:1065100002800E7407900061F0E5B5547FF5B580F8
:106520001B75A710E5CDC395704008E5B554BFF5C0
:10653000B58006E5B54440F5B575A70075A7009090
:10654000010FE0A851B80005D39552501690010EE6
:10655000E0A851B8000D95524009900110E0D39584
:10656000604002803175A710E55245516007E5CDC6
:10657000C394BF4002800EE5B54420F5B5E5B544AF
:1065800010F5B5800CE5B554DFF5B5E5B554EFF57C
:10659000B575A700802F75A710E55245516007E536
:1065A000CDC394404002800EE5B54420F5B5E5B575
:1065B0004410F5B5800CE5B554DFF5B5E5B554EFFD
:1065C000F5B575A700E56EC39409500AA2EDB34076
:1065D00005C2ED123050AE53AF547498C39F743A55
:1065E0009E400C900083E0C3945A4003026789A246
:1065F0000CB340091242647406900061F0A220B30B
:106600004008E5B54404F5B58006E5B554FBF5B59D
:10661000A20EB3500EE560D394334007E560C394F7
:10662000CC4002804190011AE0B40214120E269070
:10663000008BE075F050A4FFAEF08E5B8F5C800F96
:10664000900096E075F050A4FFAEF08E5B8F5CE595
:106650005C455B6011E5B54401F5B5741F9000829F
:10666000F0124369D20E900083E0D394014007E515
:1066700060C3941A40028002C20E9006D9E0600303
:106680001224EAA228300301B35017A228B340080D
:10669000E5B54408F5B58006E5B554F7F5B5A2288B
:1066A00092039006DDE060031225C6A229300401A2
:1066B000B35017A229B34008E5B54440F5B58006AC
:1066C000E5B554BFF5B5A22992049006E1E0600358
:1066D0001226B6A22A300501B35017A22AB34008E9
:1066E000E5B54480F5B58006E5B5547FF5B5A22A39
:1066F00092059006E5E06003122792A22B30060176
:10670000B35017A22BB34008E5B54404F5B5800695
:10671000E5B554FBF5B5A22B9206900083E0C39437
:106720005A5010E56EB40909900083E004F0756ECC
:1067300000803BE56EB40903756E00755400755317
:1067400000758D00758B00756300900082E0C39426
:106750002E5008900082E004F08006742E90008293
:10676000F0900082E0B42E06E5B554FEF5B5900039
:1067700083E0D394014007E569C394414002800956
:0C678000740E900061F0124264024A8E18
:106828000000010001400160018001A001C001E0F9
:1068380002000300039603B603D603F40400050020
:106848000512052405360548055A056C057E059090
:1068580005A805C005DE0600061406280646066ECD
:1068680006AE05CF00FF013F015F017F019F01BF19
:1068780001DF01FF02FF039503B503D503F303FF0F
:1068880004FF05110523053505470559056B057DE9
:10689800058F05A705BF05CE05F106130627064592
:1068A800066D06AD06ED05DD0FAA0FA50F9F0F9A21
:1068B8000F940F8D0F870F800F780F710F680F607F
:1068C8000F570F4E0F450F3B0F300F250F1A0F0EA6
:1068D8000F020EF50EE80EDB0ECC0EBE0EAE0E9FAE
:1068E8000E8E0E7D0E6C0E5A0E470E340E200E0CB8
:1068F8000DF70DE20DCB0DB50D9D0D850D6D0D54EC
:106908000D3A0D200D050CE90CCE0CB10C940C764B
:106918000C580C3A0C1B0BFB0BDB0BBB0B9A0B79C3
:106928000B570B350B130AF10ACE0AAB0A870A6418
:106938000A400A1C09F809D409B0098C09670943F7
:10694800091F08FB08D608B2088E086A08460823FB
:1069580007FF07DC07B9079607730751072F070DCD
:1069680006EC06CA06AA068906690649062A060A20
:1069780005EC05CD05B0059205750558053C0520C3
:10698800050504EA04CF04B5049C04820469045193
:1069980004390422040B03F403DE03C803B2039D85
:1069A800038903750361034D033B0328031603049E
:1069B80002F202E102D102C002B002A002910282F8
:1069C8000273026502570249023C022F0222021694
:1069D800020901FD01F201E601DB01D001C601BB9C
:1069E80001B101A7019D0194018B01820179017018
:1069F8000168016001580150014801410139013223
:106A0800012B0125011E01180111010B010500FFD1
:106A180000FA0FA60FA00F990F920F8B0F840F7C0F
:106A28000F740F6B0F620F580F4E0F430F380F2C58
:106A38000F1F0F120F050EF70EE80ED80EC80EB76F
:106A48000EA50E930E800E6C0E580E420E2C0E15CF
:106A58000DFD0DE40DCB0DB10D950D790D5D0D3FBF
:106A68000D200D010CE10CC00C9E0C7C0C590C3552
:106A78000C100BEA0BC40B9E0B760B4F0B260AFD72
:106A88000AD40AAA0A800A550A2A09FF09D409A8B9
:106A9800097C0950092508F908CD08A10875084A94
:106AA800081E07F307C8079D07730749072006F75D
:106AB80006CE06A6067E06570630060A05E405BF7A
:106AC800059B057705540532051004EF04CE04AE86
:106AD800048F047104530435041903FD03E203C74A
:106AE80003AD0394037B0363034B0334031E0308C2
:106AF80002F302DE02CA02B602A30291027F026D0D
:106B0800025C024C023C022C021D020E020001F241
:106B180001E401D701CA01BE01B101A6019A018FA2
:106B28000185017A01700166015D0153014A014145
:106B3800013901310129012101190112010B010457
:106B480000FD00F700F000EA00E400DE00D900D301
:106B580000CE00C900C400BF00BA00B500B100AD46
:106B680000A800A400A0009C009900950091008E48
:0C6B7800008A008700840081007E007B02
:10009E007546009007D6E4F0A3F0753000752F007A
:1000AE00754C00754D00C233D23474FE9007D8F8EB
:1000BE00E4F0E8A3F074FE9007DAF8E4F0E8A3F0B9
:1000CE0074FE9007E4F0745A9007E5F0745A9007A6
:1000DE00E6F0D235C227C237C23222750B00750A3E
:1000EE0000AE0AAF0BAC08AD09EDC39FEC9E4016F7
:1000FE0074FF126E1C75CF01780B740126F6500436
:10010E0018E436F650DB2290005DE0B4AA1C90078E
:10011E0092E0B43C159007D2E0FEA3E0FFEF4E60F4
:10012E0009741EBE0004D39F5003020243755C0087
:10013E00755B0075F8099007D2E0FEA3E0FF740727
:10014E006F4E6006740E6F4E7006743A900792F002
:10015E009007D2E0FEA3E0FF7408BE001ED39F40BE
:10016E001A7E017F089007D2E0FCA3E0FD1DBDFFC3
:10017E00011C1200038E598F5A801F9007D2E0FE89
:10018E00A3E0FF7408126E808F048E057E017F0837
:10019E00CDCCCD1200038E598F5AAE5BAF5C740C72
:1001AE00D39F74019E500302023EA2F9B3407EE536
:1001BE005C455B700375A382AE5BAF5C74016F4EE2
:1001CE00700375A300AE5BAF5C74026F4E700D9042
:1001DE0007D3E075F002A4FDACF08DA3AE5BAF5C6F
:1001EE0074036F4E700375A300AE5BAF5C7403BEF9
:1001FE0000039F5013AC59AD5AED2FFFEC3EFE900D
:10020E00008E126E63E0F5A3AE5BAF5CEFB40B092C
:10021E00EEB401057414126E1CAE5BAF5CEFB40B42
:10022E0007EEB4010375F80D785B126E900201A80B
:10023E0090005DE4F022755C00755B0075F8099026
:10024E0007D2E0FEA3E0FF7408BE001ED39F401A43
:10025E007E017F089007D2E0FCA3E0FD1DBDFF01EB
:10026E001C1200038E598F5A801F9007D2E0FEA3F6
:10027E00E0FF7408126E808F048E057E017F08CD1C
:10028E00CCCD1200038E598F5AAE5BAF5C7411D376
:10029E009F74019E5003020374A2F9B3500302032C
:1002AE0071E55C455B700375A3D2AE5BAF5C740108
:1002BE006F4E700375A300AE5BAF5C74026F4E7031
:1002CE000D9007D3E075F002A4FDACF08DA3AE5BEC
:1002DE00AF5C74036F4E700375A300AE5BAF5C74BE
:1002EE00046F4E700375A300AE5BAF5C74056F4E6A
:1002FE00700375A300AE5BAF5C74066F4E70037532
:10030E00A300AE5BAF5C74076F4E700375A300AEB7
:10031E005BAF5C74086F4E700375A300AE5BAF5C91
:10032E007408BE00039F5016AC59AD5AED2FFFEC6A
:10033E003EFE900089126E63E5A3F075A300AE5BDE
:10034E00AF5CEFB41009EEB401057414126E1CAE5E
:10035E005BAF5CEFB41007EEB4010375F80D785B7C
:10036E00126E9002029722755C00755B0075F8099B
:10037E00AE5BAF5C7417BE0004D39F500302044DF6
:10038E00A2F9B3500302044AE55C455B700375A302
:10039E00D2AE5BAF5C74016F4E700375A300AE5BA3
:1003AE00AF5C74026F4E700D9007D3E075F002A42F
:1003BE00FDACF08DA3AE5BAF5C74036F4E70037536
:1003CE00A300AE5BAF5C74046F4E700375A300AEFA
:1003DE005BAF5C74056F4E700375A300AE5BAF5CD4
:1003EE0074066F4E700375A300AE5BAF5C74076F3F
:1003FE004E700375A300AE5BAF5C74086F4E700356
:10040E0075A300AE5BAF5C7408BE00039F500C90EA
:10041E00006B126E63E5A3F075A300AE5BAF5C7468
:10042E00166F4E70057414126E1CAE5BAF5C7416B4
:10043E006F4E700375F80D785B126E9002037E227C
:10044E0090005DE0B4AB0280030204E8755C0075B9
:10045E005B0075F809AE5BAF5C7412BE007CD39F77
:10046E004078A2F9B34070E55C455B700375A382DA
:10047E00AE5BAF5C74016F4E700375A300AE5BAFE5
:10048E005C74026F4E700D9007D3E075F002A4FD00
:10049E00ACF08DA3AE5BAF5C74036F4E700375A3AF
:1004AE0000AE5BAF5C7403BE00039F5009900070FA
:1004BE00126E63E0F5A3AE5BAF5C74116F4E700508
:1004CE007414126E1CAE5BAF5C74116F4E700375BC
:1004DE00F80D785B126E90020463229007E1E4F04F
:1004EE0074649007D2F8E4F0E8A3F012037574C8B0
:1004FE009007D2F8E4F0E8A3F074FF90006BF0746C
:10050E00FF90006CF074FF90006DF0740090006529
:10051E00F074FF90006EF07400900070F074019013
:10052E000071F0900077E0B4371A900074E09000FC
:10053E006BF0900075E090006CF0900076E090000B
:10054E006DF080469007E17401F074659007D2F863
:10055E00E4F0E8A3F012037574C89007D2F8E4F043
:10056E00E8A3F0900077E0B4371A900074E09000A2
:10057E006BF0900075E090006CF0900076E09000CB
:10058E006DF0800674029007E1F09007E2E4F074DB
:10059E00669007D2F8E4F0E8A3F012037574C890E1
:1005AE0007D2F8E4F0E8A3F0900076E0B4371290AA
:1005BE000074E0900065F0900075E090006EF080A1
:1005CE00769007E27401F074679007D2F8E4F0E8D1
:1005DE00A3F012037574C89007D2F8E4F0E8A3F004
:1005EE00900076E0B43712900074E0900065F090C1
:1005FE000075E090006EF0803E74029007E2F07499
:10060E00689007D2F8E4F0E8A3F012037574C8906E
:10061E0007D2F8E4F0E8A3F0900076E0B437129039
:10062E000074E0900065F0900075E090006EF08030
:10063E000674039007E2F022E54D64046006E59926
:10064E0064FF60028031A2334004D2338027E54D2F
:10065E00600874E6254D900061F0E54C600874F07A
:10066E00254C900061F0E54DB4010280FE754D0001
:10067E00754C00C2338002C233E54D90384AF828DB
:10068E002873754D00E599B4FF03754C01E599B4D7
:10069E00FE03754C02E599B4FD03754C03E599B460
:1006AE00FC03754C04E599B4FA03754C05E599B451
:1006BE00FB06754D01124264E599B4F906754D04B9
:1006CE00124264E599D394E54007E599C394F0404E
:1006DE0002801685994E754D027E017F00E54EC350
:1006EE0094E6126E3C8E318F329007D6E4F0A3F072
:1006FE00E599D394C44007E599C394E64002802857
:10070E0085994E754D0374E5C3954EF532753100DE
:10071E00AE31AF32906828126E0BE493F8740193E9
:10072E009007D6C8F0A3C8F0D299020C5690007468
:10073E00E07005A225B3400280429007D6E0FEA3EA
:10074E00E0FF74FFBE00039F5009EFC39446EE9482
:10075E000640119007D6E0FEA3E0FFEFD3946DEEB6
:10076E00940640139007D6E0FEA3E0FF900092128D
:10077E006E63E599F0800385997380119007D6E03A
:10078E00FEA3E0FF900092126E63E599F09007D6FB
:10079E00126E4A9007D6E0FEA3E0FFEFB40106EE1C
:1007AE00B4070280030209FD900792E0B43C028078
:1007BE00030209FDA22550030208E8C29C900074B2
:1007CE00E0900130F0900075E090009FF090007680
:1007DE00E09000BFF0900077E09000E8F090007895
:1007EE00E0900094F0900079E09000DAF090007ABA
:1007FE00E09000F8F090007BE09000CCF090007C50
:10080E00E09000EAF090007DE090011AF090007EFA
:10081E00E090017EF090007FE090017FF0900080EC
:10082E00E0900180F0123B70900086E0900101F0A4
:10083E00900087E09000B8F0900088E09000B9F04A
:10084E0074639007D2F8E4F0E8A3F074AB90005D07
:10085E00F012044E90005DE4F07464F50975080022
:10086E001200E9A21F4039757201E572D394075048
:10087E002DE5729007D2F8E4F0E8A3F074AA900088
:10088E005DF0120115E572C39407500A7464F50900
:10089E007508001200E97872740126F650CC803784
:1008AE00757208E572D3940E502DE5729007D2F84A
:1008BE00E4F0E8A3F074AA90005DF0120115E57261
:1008CE00C3940E500A7464F5097508001200E97895
:1008DE0072740126F650CC0209E7C29C900130E0FA
:1008EE00900074F090009FE0900075F09000BFE0D3
:1008FE00900076F09000E8E0900077F0900094E0A1
:10090E00900078F09000DAE0900079F09000F8E036
:10091E0090007AF09000CCE090007BF09000EAE03E
:10092E0090007CF090011AE090007DF07400900031
:10093E007EF0740090007FF07400900080F074637D
:10094E009007D2F8E4F0E8A3F074AB90005DF012DB
:10095E00044E90005DE4F07464F509750800120011
:10096E00E9757201E572D394075026E5729007D2AD
:10097E00F8E4F0E8A3F074AA90005DF0120115748B
:10098E0064F5097508001200E97872740126F650B4
:10099E00D3D29C7599FB743C900792F0757208E562
:1009AE0072D3940E5026E5729007D2F8E4F0E8A3C5
:1009BE00F074AA90005DF01201157464F5097508C3
:1009CE00001200E97872740126F650D374C89007AD
:1009DE00D2F8E4F0E8A3F080FE74C89007D2F8E4F1
:1009EE00F0E8A3F0D29C754D00754C007599FB0292
:1009FE000C569007D6E0FEA3E0FFEF4E70068599E9
:100A0E0030752F009007D6E0FEA3E0FF74016F4E05
:100A1E00701BAC2FAD30AA31AB32ED2BFBEC3AFA9A
:100A2E008A068B07900092126E63E599F09007D6B6
:100A3E00126E4A9007D6E0FEA3E0FF74026F4E706E
:100A4E0021AC2FAD3074566D4C7006E54E64E660E9
:100A5E00028003124264123B70854E99754D0075EB
:100A6E004C00020C569007D6E0FEA3E0FF900092D9
:100A7E00126E63E599F09007D6126E4A9007D6E093
:100A8E00FEA3E0FFAC31AD328F028E038C068D07D4
:100A9E0090686C126E0BE493F9740193FEEAD39E88
:100AAE00EB994009854E99754D00754C00020C5618
:100ABE009007D6E0FEA3E0FF900092126E63E599D8
:100ACE00F09007D6126E4A9007D6E0FEA3E0FFEF35
:100ADE00B40006EEB401028003020C5690006DE0E5
:100AEE00D394C7400B90006DE0C394C8F54F801AA5
:100AFE0090006DE0D39463400B90006DE0C394645E
:100B0E00F54F800690006DE0F54FE54F75F002A4AD
:100B1E00FFAEF08F72EF900092126E6EEFFCE0FD62
:100B2E00EC900095126E6EEDFCE0FDEC2DB54F02D3
:100B3E008003020C470FEF900092126E6EE572FF6B
:100B4E00E0FCEF900096126E6EECFFE0FCEFC39CA3
:100B5E00B54F028003020C47E572900094126E6E40
:100B6E00E572FFE0FCEF900097126E6EECFFE0FC7A
:100B7E00EF2CB54F028003020C47E57290009812DD
:100B8E006E6EE0C3954F900074F0E572900099126E
:100B9E006E6EE0C3954F900075F0E57290009A125C
:100BAE006E6EE0C3954F900076F07400900077F073
:100BBE0074FF900078F0E57290009C126E6EE0C3A8
:100BCE00954F900079F0E57290009D126E6EE0C325
:100BDE00954F90007AF0E57290009E126E6EE0C313
:100BEE00954F90007BF0E57290009B126E6EE0C305
:100BFE00954F9007D2F8E4F0E8A3F074AB90005D47
:100C0E00F012044E7464F5097508001200E990079D
:100C1E00D2126E4A12044E7464F509750800120061
:100C2E00E99007D2126E4A12044E7599F97464F562
:100C3E00097508001200E980FE7599FF7464F509C4
:080C4E007508001200E980FEA8
:0F384A0002069002073B020A00020A73020ABE3E
:100C560022E54C903859F8282873020D699007D67A
:100C6600E0FEA3E0FF900063126E63E0F599900743
:100C7600D6126E4A9007D6E0FEA3E0FF74116F4EBF
:100C86007003754C00020D69856D99020D69900718
:100C9600D6E0FEA3E0FF900092126E63E0F599EFB6
:100CA600B40107EEB40703754C009007D6126E4ADE
:070CB600020D699007D7E071
:0F385900020C60020C63020C8E020C94020CB97C
:100CBD00903A0CF8282873855299020D5E855E993D
:100CCD00020D5E856099020D5E856499020D5E854B
:100CDD006699807D85679980788568998073856927
:100CED0099806E900026E0F5998066A234B3400796
:100CFD007599FAC2348041A224B3400575990F80CD
:100D0D00359007E1E0600A9007E1E024DCF5998079
:100D1D00169007E2E0600A9007E2E024DEF5998084
:100D2D0006900061E0F599900061E4F09007E1E430
:100D3D00F09007E2E4F0C2248017856A998012854D
:100D4D006599800D856B9980087599FC8003754CAC
:010D5D000095
:103A0C00020CC4020CCA020CD0020CD6020CDC0252
:103A1C000CE1020CE6020CEB020CF0020CF8020DAD
:0D3A2C0047020D4C020D51020D56020D5BBC
:0B0D5E009007D6126E4A8003123A394B
:03386800020D66E8
:100D690022E536255AFFAE5950010E900092126EB7
:100D790063E0F537E536255AFFAE5950010E0FBF2E
:100D890000010E900092126E63E0F538853E3AE557
:100D990037B538058537368041E538D39537401D55
:100DA900E538C395378539F0A4FFAEF0E53A8E04EE
:100DB9008F05FF126E2CED2537F536801DE537C3FB
:100DC90095388539F0A4FFAEF0E53A8E048F05FF1A
:100DD900126E2CEDF4042537F53622E538D3953714
:100DE900401DE538C395378539F0A4FFAEF0E53AE3
:100DF9008E048F05FF126E2CED2537F536801DE523
:100E090037C395388539F0A4FFAEF0E53A8E048FE3
:100E190005FF126E2CEDF4042537F5362290009863
:100E2900E0B40170E56675F00A84FF7E008F36E54F
:100E39006675F00A84ADF07C008D39753E0A7559E6
:100E490005755A24E536C394115005120D6A8006BA
:100E59009005C7E0F536E53690008BF0E56675F04C
:100E69000A84FF7E008F36E56675F00A84ADF07C52
:100E7900008D39753E0A755905755A5AE536C39478
:100E8900115005120D6A80069005FDE0F536E5362C
:100E990090001EF022900098E0B4016AE56675F0B2
:100EA9000A84FF7E008F36E56675F00A84ADF07C12
:100EB900008D39753E0A755905755A36E536C3945C
:100EC900115005120D6A80069005D9E0F536853670
:100ED9004AE56675F00A84FF7E008F36E56675F08F
:100EE9000A84ADF07C008D39753E0A755905755A2D
:100EF90048E536C394115005120D6A80069005EB3A
:100F0900E0F53685364B22E55E75F00484FF7E00F8
:100F19008F36E55E75F00484ADF07C008D39753E41
:100F290004755901755A00E536C3943F5005120DF1
:100F39006A80069001D1E0F536853628752700903C
:100F49000060E075F020A4FFAEF09000E3E08E04AD
:100F59008F05FF126E2C8D369000CBE0D3955E5035
:100F6900030210169000EFE0D3955E4010ED90015A
:100F7900D2126E6EE0F52A7529000210139000BA9C
:100F8900E0D3955E4043E5369001D2126E6EE0F5EE
:100F990037E5369001F2126E6EE0F5389000EFE019
:100FA900F404255EF5399000BAE0FE9000EFE0F414
:100FB900042EF53AE537B538058537368003120D25
:100FC900E485362A7529008041E5369001F2126ED2
:100FD9006EE0F537E536900212126E6EE0F5389044
:100FE90000BAE0F404255EF5399000CBE0FE9000EC
:100FF900BAE0F4042EF53AE537B538058537368079
:1010090003120DE485362A7529000210BD9000F2FD
:10101900E0D3955E5011E536900252126E6EE0F5FE
:101029002A7529000210BD9000BBE0D3955E50439C
:10103900E536900232126E6EE0F537E536900252CF
:10104900126E6EE0F5389000BBE0F404255EF539C8
:101059009000F2E0FE9000BBE0F4042EF53AE5378B
:10106900B538058537368003120DE485362A75298A
:10107900008041E536900212126E6EE0F537E536D2
:10108900900232126E6EE0F5389000CBE0F4042540
:101099005EF5399000BBE0FE9000CBE0F4042EF53C
:1010A9003AE537B538058537368003120DE48536BC
:1010B9002A75290022900103E0F53B753E11755907
:1010C90002755A00AE51AF52E53B75F00FA4FDAC65
:1010D900F0EDD39FEC9E4021E53B8E048F05FF1276
:1010E9006E2CED75F010A4FFAEF0E55E75F011847D
:1010F900FD7C00ED2FF53C800EE55E75F01184FF57
:101109007E00EF24F0F53C853C36E55E75F01184F0
:10111900AFF07E008F39120D6A85363DAE51AF5260
:10112900900103E075F00FA4FDACF0EDD39FEC9EA8
:101139004028755902755A10853C36120D6A853D4D
:1011490037853638AE51AF52E53B8E048F05FF1215
:101159006E578D39853B3A120DE48536287527007F
:10116900752A6475290022900103E0F53B753E114B
:10117900755902755A00AE51AF52E53B75F00FA48F
:10118900FDACF0EDD39FEC9E4021E53B8E048F052D
:10119900FF126E2CED75F010A4FFAEF0E56075F04E
:1011A9001184FD7C00ED2FF53C800EE56075F01192
:1011B90084FF7E00EF24F0F53C853C36E56075F050
:1011C9001184AFF07E008F39120D6A85363DAE511C
:1011D900AF52900103E075F00FA4FDACF0EDD39F81
:1011E900EC9E4028755902755A10853C36120D6AD5
:1011F900853D37853638AE51AF52E53B8E048F05B4
:10120900FF126E578D39853B3A120DE485362875E4
:101219002700E56A6017E56AC394FE50109000F74D
:10122900E0B402099000E5E0D3940B50028017AEB8
:1012390027AF28E56A126E3C74E78E048F05FF120A
:101249006E2C8C278D289000CDE0B40453E55E7593
:10125900F00484FF7E008F36E55E75F00484ADF0FE
:101269007C008D39753E04755901755A00E536C300
:10127900943F5005120D6A80069001D1E0F536AE13
:1012890027AF28E536126E3C74648E048F05FF1271
:101299006E2CAE27AF28EF2DFDEE3CFC8C278D2858
:1012A900752A6475290022900098E0B40146E56624
:1012B90075F00A84FF7E008F36E56675F00A84AD05
:1012C900F07C008D39753E0A755905755A00E53669
:1012D900C394115005120D6A80069005A3E0F536F6
:1012E900AE29AF2AE5362FFF50010E7464126E80C5
:1012F9008E298F2A900099E0B40146E56775F00AB6
:1013090084FF7E008F36E56775F00A84ADF07C00B6
:101319008D39753E0A755905755A6CE536C39411B0
:101329005005120D6A800690060FE0F536AE29AF1A
:101339002AE5362FFF50010E7464126E808E298FB4
:101349002A9000A8E0B40249E569C3944175F00503
:1013590084FF7E008F36E56975F00584ADF07C0069
:101369008D39753E05755906755A00E536C39413CE
:101379005005120D6A80069006A5E0F536AE29AF34
:101389002AE5362FFF50010E7464126E808E298F64
:101399002A9000EAE0B40202800302144FE55E7568
:1013A900F01584FF7E008F36E55E75F01584ADF08B
:1013B9007C008D39753E15755903755AF4E536C3A8
:1013C900940B5005120D6A8006900491E0F536E5FC
:1013D9003675F0FFA4FFAEF09000EBE08E048F05A8
:1013E900FF126E2CED900084F0E56575F078A4FF8E
:1013F900AEF074FF8E048F05FF126E2C8C598D5A36
:1014090074028C068D071200398F36AC59AD5A74A7
:1014190004FF126E578D39753E04755906755A28A1
:10142900E536C3941D5005120D6A80069006D7E073
:10143900F536AE29AF2AE5362FFF50010E74641236
:101449006E808E298F2A900097E0B4025DE5607561
:10145900F064A4FFAEF074081200398E5B8F5C74DF
:10146900058E048F05FF126E2C8D36AE5BAF5C7452
:10147900058E048F05FF126E578D39753E05755916
:1014890005755ADEE536C394135005120D6A8006B8
:10149900900683E0F536AE29AF2AE5362FFF5001D5
:1014A9000E7464126E808E298F2A9000D9E0703CE8
:1014B900900060E075F00584FF7E008F3690006033
:1014C900E075F00584ADF07C008D39753E057559E0
:1014D90005755AC0E536C3941D5005120D6A80067C
:1014E90090066FE0F536E53690008CF0229000A06A
:1014F900E0B401179007DDE0252AFFAE2950010E5F
:101509009000F4E0126E808E298F2A900118E0B4C1
:101519000114900119E0A851B8000495525007E54B
:101529005EC3955F400280129000C2E0252AFFAE9B
:101539002950010E8E298F2A802F9000A0E0B40334
:1015490016A227B3B350109007E0E0C39405A85141
:10155900B800069552400280109000C2E0252AFF8B
:10156900AE2950010E8E298F2A90009AE0B402020A
:1015790080030218F490009DE0602FE566D394463D
:10158900402890001FE0FEA3E0FF9000D8E075F02E
:1015990003A4FDACF0EFD39DEE9C400E9000FCE05F
:1015A900A851B80005D3955250030218F49000CD04
:1015B900E0B40302800302175885605A75590090F8
:1015C90000A4E0A851B800049552500E9000A5E07F
:1015D900A859B80005D3955A5003021755E5607507
:1015E900F002A4FFAEF074158E048F05FF126E2C65
:1015F9008C068D07900622126E63FEE0FFEE9000C6
:101609009CE0FEEF8E0088F0A4FFAEF074648E04B7
:101619008F05FF126E2C8C598D5A900060E075F081
:1016290018A4FFAEF09000E3E08E048F05FF126E60
:101639002C8C068D0790063A126E63AE59AF5AE0AC
:10164900126E3C74648E048F05FF126E2C8C598DBA
:101659005AE564A859B80077D3955A4072E564C32E
:10166900955AFFE49559FE8E598F5A7428BE000386
:101679009F500C755A28755900740D900061F0AE91
:1016890059AF5A90009DE0126E3C74288E048F0564
:10169900FF126E2C8C598D5AAE27AF28740A8E040E
:1016A9008F05FF126E2C8D068C07AC59AD5ACFCE23
:1016B900CF120003740A8E048F05FF126E2C8C5909
:1016C9008D5AAE27AF28126E888E278F28807DE528
:1016D90064A859B80004955A5072AE59AF5AE564D6
:1016E900126E808E598F5A7428BE00039F500C7554
:1016F9005A28755900740D900061F0AE59AF5A908F
:10170900009DE0126E3C74288E048F05FF126E2C2A
:101719008C598D5AAE27AF28740A8E048F05FF1293
:101729006E2C8D068C07AC59AD5ACFCECF12000363
:10173900740A8E048F05FF126E2C8C598D5AAE27B0
:10174900AF28EF2DFDEE3CFC8C278D280218F49074
:1017590000E5E0855EF0A4FFAEF07405126E3C74FE
:10176900071200398E598F5A9000A4E0A851B80089
:1017790004955250129000A5E075F002A4FDACF05A
:10178900EFC39DEE9C40030218F4E55E75F00B84EF
:10179900FF7E00900622126E63FEE0FFEE90009C31
:1017A900E0FEEF8E0088F0A4FFAEF074648E048F23
:1017B90005FF126E2C8C598D5A900060E075F01857
:1017C900A4FFAEF09000E3E08E048F05FF126E2CAB
:1017D9008C068D0790063A126E63AE59AF5AE01225
:1017E9006E3C74648E048F05FF126E2C8C598D5AD1
:1017F900E564A859B80077D3955A4072E564C39552
:101809005AFFE49559FE8E598F5A7428BE00039FDA
:10181900500C755A28755900740D900061F0AE5935
:10182900AF5A90009DE0126E3C74288E048F05FF1C
:10183900126E2C8C598D5AAE27AF28740A8E048FDC
:1018490005FF126E2C8D068C07AC59AD5ACFCECF41
:10185900120003740A8E048F05FF126E2C8C598DA9
:101869005AAE27AF28126E888E278F28807DE564AF
:10187900A859B80004955A5072AE59AF5AE5641286
:101889006E808E598F5A7428BE00039F500C755A6A
:1018990028755900740D900061F0AE59AF5A900047
:1018A9009DE0126E3C74288E048F05FF126E2C8CFD
:1018B900598D5AAE27AF28740A8E048F05FF126E10
:1018C9002C8D068C07AC59AD5ACFCECF12000374BC
:1018D9000A8E048F05FF126E2C8C598D5AAE27AFD4
:1018E90028EF2DFDEE3CFC8C278D28229000F8E096
:1018F900B4026AE55E75F00884FF7E008F36E55E06
:1019090075F00884ADF07C008D39753E0875590174
:10191900755AE0E536C3943F5005120D6A8006906A
:101929000291E0F53685362C752B00AE2BAF2CAC29
:1019390029AD2A12000374648E048F05FF126E2CE0
:101949008C2B8D2C900095E08C068D07126E3C74C3
:10195900648E048F05FF126E2C8C2B8D2CAE27AF55
:1019690028AC29AD2A12000374648E048F05FF1276
:101979006E2C8C278D28900095E08C068D07126EB1
:101989003C74648E048F05FF126E2C8C278D28A25F
:1019990007401DAE51AF527405BE00039F5002D2DD
:1019A90007E560D394CC4008D2017411900061F02E
:1019B9009000F7E0B402089000E5E0640B60028053
:1019C90035AE27AF28E56A126E3C74E78E048F05A1
:1019D900FF126E2C8C278D289000F8E0B40217AE08
:1019E9002BAF2CE56A126E3C74E78E048F05FF124B
:1019F9006E2C8C2B8D2C9000B7E05402601B90004C
:101A0900AEE0A851B80012D39552400DA207B3B366
:101A19005007E560C3949A40028028AE33AF3490F2
:101A290000ACE075F002A4FDACF0EF2DFDEE3CFC3E
:101A390074022DFD50010CE560BC0007D39D4003E5
:101A4900754201856034753300E5427003021B3825
:101A590090010AE0C395425003021B2A90011AE043
:101A6900C394025076E56675F00A84FF7E009005FE
:101A790092126E63E0F55A755900AE59AF5A90004B
:101A8900ADE0126E3C74648E048F05FF126E2C8CCF
:101A99005B8D5C90010AE004C395428C068D0712A8
:101AA9006E3C90010AE08E048F05FF126E2C8C5B50
:101AB9008D5CAE27AF28EF2DFDEE3CFC8C278D28E1
:101AC9009000F8E0B40212AE2BAF2CAA5BAB5CEF2E
:101AD9002BFBEE3AFA8A2B8B2C804690010AE00404
:101AE900C39542854AF0A4FFAEF090010AE08E0446
:101AF9008F05FF126E2C8C5B8D5CAE27AF28EF2D06
:101B0900FDEE3CFC8C278D289000F8E0B40212AE63
:101B19002BAF2CAA5BAB5CEF2BFBEE3AFA8A2B8B33
:101B29002C054290010AE0C395425003754200908A
:101B390000B7E05401601B9000ABE0A851B8001257
:101B4900D39552400DA207B3B35007E55EC394CCB9
:101B5900400280259000A9E075F003A4FFAEF0E5EE
:101B69003F2FFF50010E74032FFF50010EE55EBE9B
:101B79000007D39F4003754301855E3FE54370032A
:101B8900021C6B90010BE0C395435003021C5D904E
:101B9900011AE0C394025076E56675F00A84FF7E67
:101BA90000900592126E63E0F55A755900AE59AF6F
:101BB9005A9000AAE0126E3C74648E048F05FF12DD
:101BC9006E2C8C5B8D5C90010BE004C395438C06F5
:101BD9008D07126E3C90010BE08E048F05FF126E8B
:101BE9002C8C5B8D5CAE27AF28EF2DFDEE3CFC8C79
:101BF900278D289000F8E0B40212AE2BAF2CAA5B17
:101C0900AB5CEF2BFBEE3AFA8A2B8B2C80469001CA
:101C19000BE004C39543854BF0A4FFAEF090010B94
:101C2900E08E048F05FF126E2C8C5B8D5CAE27AFA6
:101C390028EF2DFDEE3CFC8C278D289000F8E0B4B0
:101C49000212AE2BAF2CAA5BAB5CEF2BFBEE3AFA80
:101C59008A2B8B2C054390010BE0C39543500375E8
:101C6900430090010DE02528FFAE2750010E8E2775
:101C79008F289000BCE0A827B80004952850099047
:101C890000BCE0F5287527009000F8E0B4020D903B
:101C990000BCE0A82BB80006952C400280099000F2
:101CA900BCE0F52C752B00229000F8E0B40102800D
:101CB90003021DBCA207B35003021DBA9000C3E082
:101CC900B40168AE27AF28AC51AD52120003743C81
:101CD9008E048F05FF126E2C9000D3E0BC00109D7E
:101CE900400D9000D5E0A827B8000495285002D2ED
:101CF90002AE27AF28AC51AD52120003743C8E04DA
:101D09008F05FF126E2C9000D3E0C3940ABC001516
:101D1900D39D40119000D5E0C39405A827B80005CC
:101D2900D3952850028002C2028068AE27AF28AC42
:101D390051AD5212000374788E048F05FF126E2C78
:101D49009000D3E0BC00109D400D9000D5E0A8277D
:101D5900B8000495285004D2028038AE27AF28ACC9
:101D690051AD5212000374788E048F05FF126E2C48
:101D79009000D3E0C3940ABC0015D39D4011900094
:101D8900D5E0C39405A827B80005D395285002804B
:101D990002C202A202B34019AE27AF289000D4E0D4
:101DA900126E3C74648E048F05FF126E2C8C278D85
:101DB900288002C202A200B34006A201B3B35009AF
:101DC900900025E4F0A3F08024AE27AF287400D357
:101DD9009F74019E400C900025E527F0A3E528F0AB
:101DE900800B74FF900025F8E4F0E8A3F09000DA86
:101DF900E0D39402400C9000C5E07006A207B3B38B
:101E09004002801AAE27AF287402126E3C8E278FCB
:101E190028AE2BAF2C7402126E3C8E2B8F2C9000A7
:101E2900C3E0B4011AAE27AF287402126E3C8E27A4
:101E39008F28AE2BAF2C7402126E3C8E2B8F2CAEDA
:101E490027AF28745E126E3C740A8E048F05FF1248
:101E59006E2C8C278D289000F8E0B40217AE2BAFBA
:101E69002C745E126E3C740A8E048F05FF126E2C60
:101E79008C2B8D2CAE27AF287402BE000AD39F404D
:101E890006752802752700AE2BAF2C7402BE000A16
:101E9900D39F4006752C02752B00900023E527F08F
:101EA900A3E528F022900060E0900392126E6EE0A4
:101EB900F540754164900060E0FE9000CEE0D39E4D
:101EC9004037E55E75F00884FF7E008F36E55E7564
:101ED900F00884ADF07C008D39753E08755903759D
:101EE9005A96E536C3941F5005120D6A8006900470
:101EF90047E0F5368536418035E55E75F00884FFA3
:101F09007E008F36E55E75F00884ADF07C008D3972
:101F1900753E08755903755AB6E536C3941F5005C1
:101F2900120D6A8006900467E0F5368536412290E5
:101F39000104E0F53B753E11755904755A00AE511F
:101F4900AF52E53B75F00FA4FDACF0EDD39FEC9ECD
:101F59004021E53B8E048F05FF126E2CED75F010C4
:101F6900A4FFAEF0E55E75F01184FD7C00ED2FF560
:101F79003C800EE55E75F01184FF7E00EF24F0F5DC
:101F89003C853C36E55E75F01184AFF07E008F39F3
:101F9900120D6A85363DAE51AF52900104E075F0DD
:101FA9000FA4FDACF0EDD39FEC9E40287559047544
:101FB9005A10853C36120D6A853D37853638AE5143
:101FC900AF52E53B8E048F05FF126E578D39853B65
:101FD9003A120DE485364075416422900104E0F51A
:101FE9003B753E11755904755A00AE51AF52E53B28
:101FF90075F00FA4FDACF0EDD39FEC9E4021E53BBD
:102009008E048F05FF126E2CED75F010A4FFAEF053
:10201900E56075F01184FD7C00ED2FF53C800EE53F
:102029006075F01184FF7E00EF24F0F53C853C36A5
:10203900E56075F01184AFF07E008F39120D6A8565
:10204900363DAE51AF52900104E075F00FA4FDACDE
:10205900F0EDD39FEC9E4028755904755A10853CC4
:1020690036120D6A853D37853638AE51AF52E53B9C
:102079008E048F05FF126E578D39853B3A120DE498
:102089008536407541649000CDE0B40479900060D4
:10209900E0FE9000CEE0D39E4037E55E75F00884FF
:1020A900FF7E008F36E55E75F00884ADF07C008D0B
:1020B90039753E08755903755A96E536C3941F500C
:1020C90005120D6A8006900447E0F5368536418091
:1020D90035E55E75F00884FF7E008F36E55E75F0A4
:1020E9000884ADF07C008D39753E08755903755A21
:1020F900B6E536C3941F5005120D6A800690046731
:10210900E0F53685364122900098E0B4013BE5665A
:1021190075F00A84FF7E008F36E56675F00A84AD96
:10212900F07C008D39753E0A755905755A12E536E8
:10213900C394115005120D6A80069005B5E0F53675
:10214900E5412536C39464F541900099E0B4013B1B
:10215900E56775F00A84FF7E008F36E56775F00A3A
:1021690084ADF07C008D39753E0A755905755A7E26
:10217900E536C394115005120D6A8006900621E0D8
:10218900F536E5412536C39464F541E5402541F529
:10219900359000A0E0B402109007DCE02535FE90F0
:1021A90000F4E0F4042EF5359000F7E0D3940140F3
:1021B90040E56AC394E7501D74E7C3956AFE90072A
:1021C900DEE08E00F5F0E884FF7E008F36E53525E8
:1021D90036F535801CE56AC394E7FE9007DEE08E8C
:1021E90000F5F0E884FF7E008F36E535C39536F5B6
:1021F90035A2074006E5402464F535E535D39464F6
:102209004009E535C39464F53580037535009000C0
:10221900D0E0C3953550069000D0E0F53522D200C4
:1022290090008AE0A851B800049552504190008A64
:10223900E0A851B800049552500375350F90008AF3
:10224900E004A851B800049552500375350A90006E
:102259008AE02402A851B800049552500575350545
:10226900C20090008AE060067409900061F0C237EC
:102279007E017F009000D6E0126E3C9000E5E08E72
:10228900048F05FF126E2CE55EBC0017D39D401329
:102299009000DFE0B40204D2378002C200740A90D1
:1022A9000061F09000D7E0C3956650159000E9E011
:1022B900A851B8000495525002C200740B900061F5
:1022C900F0E566C39464501D90012FE0600D900104
:1022D9002FE0A851B80006955240028008C2007448
:1022E9000B900061F0A2004003753505900118E0DC
:1022F900B40114900119E0A851B80004955250078F
:10230900E55EC3955F400280089000C1E0F5358025
:102319003A9000A0E0B40306A227B3B34002802B91
:102329009007E0E0C39405A851B800049552500CF9
:102339009000C1E0F535740C900061F09007E0E081
:10234900A851B8000495525002C20085356B90001F
:1023590092E02535FE900060E075F01E84FC7F0058
:10236900EE2CF53522900060E075F00584FF7E00C3
:102379008F36900060E075F00584ADF07C008D39F2
:10238900753E05755903755AD69000E3E01475F04A
:102399000584FF7E00E536BE00039F5005120D6AD5
:1023A900800BE536900468126E6EE0F536E53690DE
:1023B90007DFF09007DFE0FE9000D2E0C39E5008EF
:1023C9009000D2E09007DFF022E56675F00A84FFFD
:1023D9007E00900592126E63E0F545E545D394645D
:1023E9004010E545C3946475F00F84FF7E008F4566
:1023F90080037545009000B5E02545F5452290001C
:10240900CDE0C3940350269007CCE0FEA3E0FF740F
:1024190004120039E55E126E3C740F8E048F05FFBD
:10242900126E2C9007CAECF0A3EDF080249007CC33
:10243900E0FEA3E0FF7404120039E560126E3C74FB
:102449000F8E048F05FF126E2C9007CAECF0A3EDD6
:10245900F09000A8E0B40262E569C3944175F00503
:1024690084FF7E008F36E56975F00584ADF07C0048
:102479008D39753E05755906755A14E536C3941795
:102489005005120D6A80069006B9E0F5369007CA24
:10249900E0FEA3E0FF740A8E048F05FF126E2CE59F
:1024A900368C068D07126E3C740A8E048F05FF1256
:1024B9006E2C9007CAECF0A3EDF09007CAE0FEA3DA
:1024C900E0FF9007D0E0FCA3E0FDEDD39FEC9E4038
:1024D9000F9007D0E0F8A3E09007CAC8F0A3C8F0AE
:1024E900229006D9E090386BF8282873804C8552E1
:1024F9007280479000E5E0855EF0A4FFAEF07408B5
:102509001200398F728033856072802E85667280E1
:10251900298567728024856872801F856972801A8F
:10252900856A7280158565728010856472800B8555
:0A2539006B728006900026E0F57238
:10386B000224F50224F70224FC022510022515027E
:10387B00251A02251F02252402252902252E0225A1
:07388B003302253802253D40
:102543009006DAE0FE9006DBE0D39E404B9006D97E
:10255300E0B404189006DBE0C395725002D22890D1
:1025630006DAE0D395724002C228802A9006DAE0A8
:10257300C3957250099006DBE0D395725002800236
:10258300D2289006DAE0D3957250099006DBE0C3B7
:1025930095725002C228802A9006DAE0D3957240E1
:1025A300099006DBE0C3957240028002C2289006C0
:1025B300DAE0C3957240099006DBE0D395724002DE
:1025C300D228229006DDE0903892F8282873804CB8
:1025D30085527280479000E5E0855EF0A4FFAEF07F
:1025E30074081200398F728033856072802E85667D
:1025F3007280298567728024856872801F8569725D
:10260300801A856A72801585657280108564728070
:0C2613000B856B728006900026E0F572CB
:103892000225D10225D30225D80225EC0225F10208
:1038A20025F60225FB02260002260502260A02262A
:0738B2000F02261402261983
:10261F009006DEE0FE9006DFE0D39E405F9006DD81
:10262F00E0B404189006DFE0C395725002D22990EF
:10263F0006DEE0D395724002C229803E9006DEE0AE
:10264F00C3957250099006DFE0D395725002800255
:10265F00D2299006DEE0D3957250099006DFE0C3D1
:10266F0095725002C2299006DDE0B401099000F185
:10267F00E0D3956050028002C229802A9006DEE0E6
:10268F00D3957240099006DFE0C395724002800235
:10269F00C2299006DEE0C3957240099006DFE0D3B1
:1026AF0095724002D229229006E1E09038B9F828BD
:1026BF002873804C85527280479000E5E0855EF06C
:1026CF00A4FFAEF074081200398F728033856072E8
:1026DF00802E856672802985677280248568728056
:1026EF001F856972801A856A7280158565728010E0
:1026FF00856472800B856B728006900026E0F57200
:1038B9000226C10226C30226C80226DC0226E1022C
:1038C90026E60226EB0226F00226F50226FA022651
:0738D900FF0227040227098A
:10270F009006E2E0FE9006E3E0D39E404B9006E198
:10271F00E0B404189006E3E0C395725002D22A90F9
:10272F0006E2E0D395724002C22A802A9006E2E0C8
:10273F00C3957250099006E3E0D395725002800260
:10274F00D22A9006E2E0D3957250099006E3E0C3D7
:10275F0095725002C22A802A9006E2E0D395724009
:10276F00099006E3E0C3957240028002C22A9006E8
:10277F00E2E0C3957240099006E3E0D39572400200
:10278F00D22A229006E5E09038E0F8282873804C92
:10279F0085527280479000E5E0855EF0A4FFAEF0B1
:1027AF0074081200398F728033856072802E8566AF
:1027BF007280298567728024856872801F8569728F
:1027CF00801A856A728015856572801085647280A3
:0C27DF000B856B728006900026E0F572FE
:1038E00002279D02279F0227A40227B80227BD02B4
:1038F00027C20227C70227CC0227D10227D60227D8
:07390000DB0227E00227E5CE
:1027EB009006E6E0FE9006E7E0D39E404B9006E5B0
:1027FB00E0B404189006E7E0C395725002D22B9018
:10280B0006E6E0D395724002C22B802A9006E6E0E2
:10281B00C3957250099006E7E0D39572500280027F
:10282B00D22B9006E6E0D3957250099006E7E0C3F1
:10283B0095725002C22B802A9006E6E0D395724027
:10284B00099006E7E0C3957240028002C22B900606
:10285B00E6E0C3957240099006E7E0D3957240021B
:10286B00D22B229006E9E0903907F8282873804C88
:10287B0085527280479000E5E0855EF0A4FFAEF0D4
:10288B0074081200398F728033856072802E8566D2
:10289B007280298567728024856872801F856972B2
:1028AB00801A856A728015856572801085647280C6
:0C28BB000B856B728006900026E0F57221
:1039070002287902287B022880022894022899023B
:10391700289E0228A30228A80228AD0228B202285E
:07392700B70228BC0228C111
:1028C7009006EAE0FE9006EBE0D39E404B9006E9C7
:1028D700E0B404189006EBE0C395725002D22C9036
:1028E70006EAE0D395724002C22C802A9006EAE0FD
:1028F700C3957250099006EBE0D39572500280029F
:10290700D22C9006EAE0D3957250099006EBE0C30B
:1029170095725002C22C802A9006EAE0D395724045
:10292700099006EBE0C3957240028002C22C900624
:10293700EAE0C3957240099006EBE0D39572400236
:10294700D22C229006EDE090392EF8282873804C7F
:1029570085527280479000E5E0855EF0A4FFAEF0F7
:1029670074081200398F728033856072802E8566F5
:102977007280298567728024856872801F856972D5
:10298700801A856A728015856572801085647280E9
:0C2997000B856B728006900026E0F57244
:10392E0002295502295702295C02297002297502C3
:10393E00297A02297F02298402298902298E0229E5
:07394E009302299802299D54
:1029A3009006EEE0FE9006EFE0D39E404B9006EDDE
:1029B300E0B404189006EFE0C395725002D22D9054
:1029C30006EEE0D395724002C22D802A9006EEE017
:1029D300C3957250099006EFE0D3957250028002BE
:1029E300D22D9006EEE0D3957250099006EFE0C326
:1029F30095725002C22D802A9006EEE0D395724064
:102A0300099006EFE0C3957240028002C22D900642
:102A1300EEE0C3957240099006EFE0D39572400251
:102A2300D22D229006F1E0903955F8282873804C76
:102A330085527280479000E5E0855EF0A4FFAEF01A
:102A430074081200398F728033856072802E856618
:102A53007280298567728024856872801F856972F8
:102A6300801A856A7280158565728010856472800C
:0C2A73000B856B728006900026E0F57267
:10395500022A31022A33022A38022A4C022A51024B
:103965002A56022A5B022A60022A65022A6A022A6C
:073975006F022A74022A7997
:102A7F009006F2E0FE9006F3E0D39E404B9006F1F5
:102A8F00E0B404189006F3E0C395725002D22E9072
:102A9F0006F2E0D395724002C22E802A9006F2E031
:102AAF00C3957250099006F3E0D3957250028002DD
:102ABF00D22E9006F2E0D3957250099006F3E0C340
:102ACF0095725002C22E802A9006F2E0D395724082
:102ADF00099006F3E0C3957240028002C22E900661
:102AEF00F2E0C3957240099006F3E0D3957240026D
:102AFF00D22E229006F5E090397CF8282873804C6E
:102B0F0085527280479000E5E0855EF0A4FFAEF03D
:102B1F0074081200398F728033856072802E85663B
:102B2F007280298567728024856872801F8569721B
:102B3F00801A856A7280158565728010856472802F
:0C2B4F000B856B728006900026E0F5728A
:10397C00022B0D022B0F022B14022B28022B2D02D3
:10398C002B32022B37022B3C022B41022B46022BF3
:07399C004B022B50022B55DA
:102B5B009006F6E0FE9006F7E0D39E404B9006F50C
:102B6B00E0B404189006F7E0C395725002D22F9090
:102B7B0006F6E0D395724002C22F802A9006F6E04B
:102B8B00C3957250099006F7E0D3957250028002FC
:102B9B00D22F9006F6E0D3957250099006F7E0C35A
:102BAB0095725002C22F802A9006F6E0D3957240A0
:102BBB00099006F7E0C3957240028002C22F90067F
:102BCB00F6E0C3957240099006F7E0D39572400288
:102BDB00D22F229006F9E09039A3F8282873804C65
:102BEB0085527280479000E5E0855EF0A4FFAEF061
:102BFB0074081200398F728033856072802E85665F
:102C0B007280298567728024856872801F8569723E
:102C1B00801A856A72801585657280108564728052
:0C2C2B000B856B728006900026E0F572AD
:1039A300022BE9022BEB022BF0022C04022C09025E
:1039B3002C0E022C13022C18022C1D022C22022C7A
:0739C30027022C2C022C311D
:102C37009006FAE0FE9006FBE0D39E404B9006F923
:102C4700E0B404189006FBE0C395725002D23090AE
:102C570006FAE0D395724002C230802A9006FAE065
:102C6700C3957250099006FBE0D39572500280021B
:102C7700D2309006FAE0D3957250099006FBE0C374
:102C870095725002C230802A9006FAE0D3957240BE
:102C9700099006FBE0C3957240028002C23090069D
:102CA700FAE0C3957240099006FBE0D395724002A3
:102CB700D230229006FDE09039CAF8282873804C5C
:102CC70085527280479000E5E0855EF0A4FFAEF084
:102CD70074081200398F728033856072802E856682
:102CE7007280298567728024856872801F85697262
:102CF700801A856A72801585657280108564728076
:0C2D07000B856B728006900026E0F572D0
:1039CA00022CC5022CC7022CCC022CE0022CE502E8
:1039DA002CEA022CEF022CF4022CF9022CFE022D06
:0739EA0003022D08022D0D60
:102D13009006FEE0FE9006FFE0D39E404B9006FD3A
:102D2300E0B404189006FFE0C395725002D23190CC
:102D330006FEE0D395724002C231802A9006FEE07F
:102D4300C3957250099006FFE0D39572500280023A
:102D5300D2319006FEE0D3957250099006FFE0C38E
:102D630095725002C231802A9006FEE0D3957240DC
:102D7300099006FFE0C3957240028002C2319006BB
:102D8300FEE0C3957240099006FFE0D395724002BE
:102D9300D23122AE2DAF2E74F5D39F74019E40081D
:102DA300782D126E90022EB0752E01752D00AE5146
:102DB300AF52E545BE000DD39F40099000C7E0D355
:102DC300954640028023754600E545C39552F5724A
:102DD3009000CAE0D395444008E5442572F5448049
:102DE300069000CAE0F544800205469000A3E0D3B4
:102DF3009560401CE55EC3955F4015AE51AF52E54B
:102E030045BE00039F50099000C8E0D39547400298
:102E1300806E9007E3E0A851B80004955250037503
:102E230049009007E3E0A851B8000BD39552400640
:102E3300E5529007E3F0E5497041E552C39545F546
:102E430072E572D3940540037572059000C9E0C31F
:102E530095445007E572C3954440028009E544C395
:102E63009572F54480069000C9E0F5449000C9E0EE
:102E7300D3954440069000C9E0F5447547008002AD
:102E83000547E54970169000A3E0C39560500DE532
:102E9300452405A851B8000695524002800F9000C2
:102EA300B6E0F54475490174789007E3F022AE2D3E
:102EB300AF2E74E9D39F74039E4008782D126E9051
:102EC30002304F752E01752D00754432A232402A0F
:102ED3007544199000B6E075F002A4FFAEF0E54624
:102EE300BE0006D39F4002D232054675490374786B
:102EF3009007E3F075480002303EAE51AF52E5450E
:102F03006F4E700302303EE545BE000DD39F40096E
:102F13009000C7E0D395464002800F754600E5490F
:102F2300C394035003754419800DE545C39552F5C9
:102F330072E5462572F5469000A3E0D39560400EF6
:102F43009007E3E0A851B80007D395524002800CE4
:102F530005489000B6E0B54803754900E549B40358
:102F630006A207B3B34002800A0548E548B43C0310
:102F7300754902E549B402299007E3E0A851B80076
:102F83000ED395524009E5529007E3F0754800903F
:102F930000A3E0C39560500975480074789007E377
:102FA300F0E549705A9000A3E0D39560401CE55EBC
:102FB300C3955F4015AE51AF52E545BE00039F5028
:102FC300099000C8E0D39547400280087547007513
:102FD300444B8028E552C39545F572E572D39405B9
:102FE30040037572059000A3E0D395604008E54760
:102FF3002572F5478006E5472406F547754800E541
:103003004970169000A3E0C39560500DE545240573
:10301300A851B80006955240028003754901E5495D
:10302300B4011875441905489000B6E0B548067513
:10303300490275480074789007E3F0E54475F00A97
:10304300A4FFAEF09007D4EEF0A3EFF022E56E906C
:1030530039F1F828287390009BE0700302327790CF
:1030630000D1E0B40102800302319290005EE0B52A
:103073005D02800302318F7E017F00E5BE126E3C4C
:10308300E5BD2FFF50010E8E598F5A7410126E3CFE
:10309300900089E08E048F05FF126E2C9007D8EC08
:1030A300F0A3EDF074FFBC00039D500B74FF900779
:1030B300D8F8E4F0E8A3F0E56A600FE56AC394FE8C
:1030C30050089000F7E06402600280649000E5E03D
:1030D300B40B1F9007D8E0FEA3E0FF74E7126E3C29
:1030E300E56A8E048F05FF126E2C9007D8ECF0A3CF
:1030F300EDF09000E5E0D3940B40089000CDE06440
:10310300046002802B9007D8E0FEA3E0FF9007DA6B
:10311300E0FCA3E0FDEFD39DEE9C400D126E889082
:1031230007D8EEF0A3EFF080079007D8E4F0A3F000
:1031330090009BE0B4021E9007D8E0FEA3E0FF904E
:1031430007E4E02FFF50010E74011200399007D8F5
:10315300EEF0A3EFF09007D8E0FEA3E0FF9007E4C2
:10316300E0BE0008D39F4004D2358002B2359007F9
:10317300D9E09007E4F09000CDE064016006A23549
:10318300B3B3400280069007D9E0F55E023275D2F0
:10319300357E017F00E5BE126E3CE5BD2FFF500179
:1031A3000E8E598F5A7410126E3C900089E08E0473
:1031B3008F05FF126E2C9007D8ECF0A3EDF0E56AB3
:1031C300600FE56AC394FE50089000F7E064026064
:1031D3000280649000E5E0B40B1F9007D8E0FEA3E3
:1031E300E0FF74E7126E3CE56A8E048F05FF126EF2
:1031F3002C9007D8ECF0A3EDF09000E5E0D3940B0E
:1032030040089000CDE064046002802B9007D8E072
:10321300FEA3E0FF9007DAE0FCA3E0FDEFD39DEE11
:103223009C400D126E889007D8EEF0A3EFF0800754
:103233009007D8E4F0A3F090009BE0B4021E90073F
:10324300D8E0FEA3E0FF9007E4E02FFF50010E74E7
:10325300011200399007D8EEF0A3EFF09007D9E000
:103263009007E4F09000CDE0640160069007D9E098
:10327300F55E8003755E00900097E07006756E0141
:1032830002305075BB18023845900097E070030276
:1032930033FD7E017F00E5BE126E3CE5BD2FFF507E
:1032A300010E8E598F5A9000DDE0B4010F7E0F7F1F
:1032B300FFAC59AD5A126E888E598F5A900102E0B5
:1032C300B40245AE59AF5A90002FE0FCA3E0FDEDE8
:1032D300D39FEC9E400A90002FE559F0A3E55AF0E6
:1032E300AE59AF5A900031E0FCA3E0FDEFD39DEE61
:1032F3009C400A900031E559F0A3E55AF0AE59AF6E
:103303005A74041200398F60900102E0704CAE5978
:10331300AF5A90002FE0FCA3E0FDEFD39DEE9C405D
:1033230009126E888E598F5A8006755A0075590096
:10333300AE59AF5A7410126E3C900086E08E048F23
:1033430005FF126E2C8C598D5A74FFBC0009D39D56
:103353004005855A6080037560FE9000CDE0B4019E
:103363000280030233FBA207B3B3500E9000A1E027
:10337300A851B80005D39552500280719000DEE049
:103383008560F0A4FFAEF074648E048F05FF126EA7
:103393002C8C598D5AE56A6016E56AC394FE500F6A
:1033A3009000F7E0B402089000E5E0640B6002804F
:1033B30017AE59AF5A74E7126E3CE56A8E048F0557
:1033C300FF126E2C8C598D5AAE59AF5A9007D8E024
:1033D300FCA3E0FDEDD39FEC9E4005855A5E800B78
:1033E300A235B340069007D9E0F55E800BA235B352
:1033F30040069007D9E0F55E800375600090009A5F
:10340300E07006756E0202305075BB1902384590A4
:10341300009AE070030234B2E55DD3955040030295
:1034230034B090002DE0FEA3E0FFE564126E8090BF
:10343300002DEEF0A3EFF07E017F00E5BE126E3C9F
:10344300E5BD2FFF50010E8E598F5A900107E07092
:1034530013740A126E3C74518E048F05FF126E2C86
:103463008D648019AE59AF5A740A126E3C8F048E64
:10347300057E017F95CDCCCD126D2A8F64E564D393
:103483009464400375646490002DE0FEA3E0FFE5BF
:10349300642FFF50010E90002DEEF0A3EFF090008B
:1034A3009EE0048E048F05FF126E2C8D64800375DD
:1034B30064329000EAE07006756E0302305075BB0B
:1034C300130238459000EAE0604A7E017F00E5BEC2
:1034D300126E3CE5BD2FFF50010E8E598F5A7404B6
:1034E3001200398F659000ECE08565F0A4FDACF027
:1034F3007464FF126E2C8D659000EBE08565F0A47B
:10350300FFAEF074FF8E048F05FF126E2CED90005A
:1035130085F08003756500900098E07006756E0471
:1035230002305075BB17023845900098E0B4010291
:1035330080030235C07E017F00E5BE126E3CE5BD0F
:103543002FFF50010E8E598F5A9007E5E0601990B6
:1035530007E5E0149068B012008CE493FC740193C7
:10356300FDEDC39FEC9E400280069007E5E014F05A
:103573009007E5E0C394B3501DAE59AF5A9007E5E9
:10358300E0049068B012008CE493FC740193FDEFA7
:10359300C39DEE9C400280069007E5E004F090078F
:1035A300E5E0FE9000BEE08E0088F0A4FFAEF0746C
:1035B300648E048F05FF126E2C8D66800375660082
:1035C300900099E07006756E0502305075BB1602C7
:1035D3003845900099E0B4010280030236697E0108
:1035E3007F00E5BE126E3CE5BD2FFF50010E8E59E4
:1035F3008F5A9007E6E060199007E6E014906A1A84
:1036030012008CE493FC740193FDEDC39FEC9E4088
:103613000280069007E6E014F09007E6E0C394B357
:10362300501DAE59AF5A9007E6E004906A1A120093
:103633008CE493FC740193FDEFC39DEE9C400280E8
:10364300069007E6E004F09007E6E0FE9000C4E091
:103653008E0088F0A4FFAEF074648E048F05FF1211
:103663006E2C8D67800375670075BB1F0238457E1E
:10367300017F00E5BE126E3CE5BD2FFF50010E8EAB
:10368300598F5A7409126E3C74E68E048F05FF122B
:103693006E2C8D699000A0E07006756E07023050A5
:1036A30075BB150238459000A0E070030237C47E55
:1036B300017F00E5BE126E3CE5BD2FFF50010E8E6B
:1036C300598F5A74041200398F689000A0E0B40136
:1036D300159000F4E08568F0A4FFAEF074071200C3
:1036E30039EF9007DDF09000A0E0B402159000F4EC
:1036F300E08568F0A4FFAEF07407120039EF90077D
:10370300DCF09000A0E0B4030280030237A790002E
:10371300E1E0701CE568C394195002D227E568D331
:1037230094644002C2279000C0E09007E0F08063F9
:103733009000C0E070349000F4E08568F0A4FFAE20
:10374300F074FF8E048F05FF126E2CED9007E0F0EE
:10375300AE51AF52741EBE0006D39F4002D227E57E
:1037630060D394E54002C2278029E568C3940A50D8
:103773000DAE51AF52741EBE0004D39F500280029F
:10378300D227E560D394E54002C2279000C0E090C1
:1037930007E0F09007E0E0C3940550067405900736
:1037A300E0F0C2369000A0E0B40414E568C39419B5
:1037B3005002D236E568D394324002C236C2278023
:1037C300037568009000F7E07006756E08023050CC
:1037D30075BB14806D9000F7E060567E017F00E5B5
:1037E300BE126E3CE5BD2FFF50010E8E598F5AEF6E
:1037F300D39421EE940E4005756AFF8015AE59AF40
:103803005A7410126E3C74E38E048F05FF126E2CF3
:103813008D6AE56A75F00BA4FFAEF09000E5E08ECB
:10382300048F05FF126E2C9007DAECF0A3EDF08005
:1038330003756A0090009BE0600575BB1A800375F1
:02384300BB18B0
:1039F10002305902328C0234120234C702352C02D1
:0B3A010035D50236720236A90237D814
:05384500056ED2EC222B
:096E6E002582F582500205832201
:0F008C0025E050020583258250020583F582226C
:106E0B00EF2F500205832582F582E5833E2EF58315
:016E1B002254
:106E8000CFC39FFF50011E22C3EF9DFFEE9CFE2249
:086E90000806B60002180622F4
:0D6E4A00A3E004F07006120049E004F022FD
:0E003900048007C3CE13CECF13CFD5E0F6223E
:106D2A00BC000FBE0008ED8FF084FFADF022E4FE38
:106D3A00FF22BE000DEF60FE54F0606F20E70302F1
:106D4A006DE0EAC0E0EBC0E078017A0075F001EE90
:106D5A0020E710EF25E0FFEE33FE0AC5F023C5F069
:106D6A0030E7F0EA5407F9096A7A007B0060010803
:106D7A00C3EC9E40167004ED9F4010ED9FFDEC9E03
:106D8A00FCE5F0CA4ACA03F5F08005E5F003F5F020
:106D9A00C3EE13FEEF13FFD9D77908CACBCAD8D0EE
:106DAA00EAFEEBFFD0E0FBD0E0FA22EC8FF084FCA5
:106DBA00ED54F045F0C48FF084FEEDC454F045F074
:106DCA00C48FF084FDEEC4FE54F02DFFEE540F3C48
:106DDA00FEADF07C0022790078008FF0EC7E08206E
:106DEA00E70DC3CD33CD33C933C9C833C8DEF08408
:106DFA0049F9E5F08FF0BE00E6FD7C00E9FFE8FE08
:016E0A002265
:0E6E3C00F88FF0A4FFE5F0CE88F0A42EFE2221
:10000300EF8DF0A4F9A8F0EF8CF0A428F8EE8DF0B2
:06001300A428FEE9FF2213
:106E1C00600D782B026E26007830D8FED5E0F82273
:106E2C00EEC0E07E00126D2AEFFDEEFCD0E0FE22FB
:0C6E5700EEC0E07E00126D2AD0E0FE22AA
:03001B0002001EC2
:0300530002005652
:03009B00020071EF
:03000000026E7716
:096E770075817475D0000244AC71
:0B6E6300E5822FF582E5833EF58322D7
:0A0049000582D5820215831582227C
:10001E00C0E0C0F0C083C082C0D075D00012445082
:0B002E00D0D0D082D083D0F0D0E032E0
:10005600C0E0C0F0C083C082C0D075D00012445347
:10006600D0D0D082D083D0F0D0E032C0E0C0F0C093
:1000760083C082C0D075D000124475D0D0D082D053
:0600860083D0F0D0E0324F
:00000001FF
